:1080000000000020BD870000758500008585000008
:108010008585000085850000858500008585000038
:108020008585000085850000858500008585000028
:10803000858500008585000085850000759A000013
:108040008585000085850000858500008585000008
:1080500085850000858500008585000085850000F8
:1080600085850000858500008585000085850000E8
:1080700085850000858500008585000085850000D8
:1080800085850000858500008585000085850000C8
:1080900085850000858500008585000085850000B8
:1080A00085850000858500008585000085850000A8
:1080B0008585000085850000858500008585000098
:1080C0008585000085850000858500008585000088
:1080D0008585000085850000858500008585000078
:1080E0008585000085850000858500008585000068
:1080F0008585000085850000858500003596000097
:108100008585000085850000858500008585000047
:108110008585000085850000858500008585000037
:108120008585000085850000858500008585000027
:10813000858500008585000041F8000085850000E8
:108140008585000085850000858500008585000007
:1081500085850000858500008585000085850000F7
:10816000D5FD00008585000085850000858500001F
:1081700085850000858500008585000085850000D7
:1081800085850000858500008585000085850000C7
:1081900085850000858500008585000085850000B7
:1081A0008DEC0000BDEC0000858500008585000099
:1081B0008585000085850000858500008585000097
:1081C0008585000085850000858500008585000087
:1081D0008585000085850000858500008585000077
:10840000FFFFFFFFFFFFFFFFFFFFFFFF7EFFFFFFFD
:1084100010B5054C237833B9044B13B10448AFF3BE
:1084200000800123237010BDA800FF1F0000000082
:10843000842C01000C4B43B10C480D4910B5AFF32F
:1084400000800C48036823B910BD0A48036833B99B
:108450007047094B002BF7D0BDE810401847064B7A
:10846000002BF5D0184700BF00000000842C01004D
:10847000AC00FF1FA800FF1F0000000000280346FB
:10848000B8BF00F11F035B11012B2BD0022B15D0BD
:1084900003B170471D4A434203F01F03D2F8801115
:1084A00000F01F0058BF5842012303FA00F00143B7
:1084B000C2F880111368184310607047134A434292
:1084C00003F01F03D2F8881100F01F0058BF584274
:1084D000012303FA00F00143C2F88811936818439E
:1084E00090607047094A414201F01F0100F01F00EF
:1084F00058BF4842D2F8841103FA00F00143C2F891
:108500008411536818435060704700BF00E100E0D9
:1085100080281ADC40280FDC20281FDC434203F0AF
:108520001F0300F01F00124A58BF5842012303FAEC
:1085300000F0C2F88000704700F01F0001230C4AD1
:1085400003FA00F0C2F88800704700F01F00012312
:10855000074A03FA00F0C2F88C00704700F01F00D1
:108560000123034A03FA00F0C2F88400704700BFF9
:1085700000E100E0684620F007018D4601B401BC2F
:1085800085467047684620F007018D4601B4FFBE5E
:1085900001BC8546704700BF4FF0E020F0B5364B78
:1085A000364A374CC0F8084D41F244053549364F3C
:1085B0004CF220544DF628164FF4E970D481D68140
:1085C00041F23804108059511A59304E304831491F
:1085D00042F4D0521A515E5141F248042E4E1A59BB
:1085E00022F00F0242F002021A5141F204024FF04F
:1085F000240E9C5844F480349C501D6825F40025BA
:108600001D60856C3D408564C46C80253C40C4641D
:1086100081F801E03570985820F001009850A223AD
:108620000B70CB78032403F01F030020CB700A46A5
:108630000C71487193799807FCD5164A9379D9063D
:10864000FCD4144A937903F00C03082BFAD140238D
:10865000104953718B7903F00C03082BFAD10D4AA2
:1086600093795B06FCD522230A4913708B7903F0BA
:108670000C030C2BFAD1F0BD007004400020054023
:108680000080000000003301FFF8FFFE000013012E
:1086900000900440004006400050064080F31188DE
:1086A000704700BFF0B41A4D1A4C2B691A4E1B4A82
:1086B0001B481C4923F0807323F4E06341F2140744
:1086C00043F4E0632B610025E55104F582531C68F7
:1086D00044F004041C60336823F0784323F0010362
:1086E0003360137803F08C0343F050031370537816
:1086F00003F09C0343F040035370937803F0EC03C2
:108700009370857081F8145385F31188F0BC70471D
:10871000009004400070044000D0004000D00740AA
:1087200000E0074000E100E0E2B140EA010313F09D
:10873000030F07D1032A05D951F8043B40F8043B45
:10874000043AF1E7DB0707D4012A05D931F9023BE6
:1087500020F8023B023AE7E711F8013B00F8013B41
:10876000013AE1E7704700BF704700BF884201D07F
:1087700002B1D9E7704700BF10B50C4C24B913E023
:1087800070B9A3688BB10C34216860680029F7D0F8
:108790008142A268F7D0002AF5D0FFF7C5FFF2E7C3
:1087A000A268002AEFD0F8E710BD10BD9C2D010093
:1087B000704700BF704700BF704700BF10B5FFF79C
:1087C000F7FF1D4CFFF7E8FE2046002807D085463E
:1087D00081B04FF000006FEA0000009001B0174B2D
:1087E000174AD21A0AD0002113F0030012D1032A2B
:1087F00010D9043A43F8040B002AF5D1FFF7BCFF67
:10880000FFF7DAFF0F49002009F012FD0E4B186048
:108810008047FEE713F0010007D1012A05D0023A94
:1088200023F8020B002ADFD1E8E7013A03F8011B25
:10883000002AD9D1E2E700BF00000020A800FF1FF6
:108840007451FF1FC400FF1F4403FF1F08B5FFF74B
:10885000B5FF00BF70B40D4B00220726082501208C
:1088600002214FF4FA741E705D7158709A701A717B
:108870009A711A755A759A75DA75D9701C62986072
:108880001A619A61DA61D96070BC70472003FF1FDA
:10889000304B314AF0B506209A65FA260A2508279A
:1088A000C8244FF4967247F230515E61DD614FF497
:1088B0007A664FF4FA7583F8250083F8297005204D
:1088C0004FF4FA671C669A6401240022D9654FF4BC
:1088D0007A711E605E60DE639D601D635D631C6275
:1088E00083F8244083F82C405985D9644FF4827E64
:1088F00040F2FF76D86018619F619F6378254FF43E
:10890000C87483F8262083F8272083F8282083F86A
:108910002D20A3F8402083F842205A6483F8542085
:10892000196547F6FF7183F8642083F82E2083F8D9
:10893000692083F86A20A3F86E00A3F86CE0A3F81E
:1089400072609D67DC67A3F87010A3F87410A3F839
:108950007610F0BD9C02FF1FC0B85900364B374956
:1089600041F23802F0B49858354C364F364E374DF8
:1089700040F4007098504FF4E0602060E060985838
:1089800040F4806098504FF481744FF480700C650F
:10899000C8607C6924F480147C610C6D2C4F24F039
:1089A00020040C650C6D44F002040C650C6D24F081
:1089B00001040C659958274C41F400619950F0630B
:1089C0003064995841F480519950696941F04001EF
:1089D0006961296821F040012960B8619D581E4FE6
:1089E0001E4945F400559D50626942F004026261DF
:1089F000226806F5005641F22C0522F0040222609E
:108A0000B0605859B7F8722040F48050585191F82E
:108A1000213043F0800381F8213091F82130C2F3F6
:108A2000032443F04003D2B281F821304C700A7025
:108A30000020F0BC704700BF0070044000A004405C
:108A40000090044040F00F4000B00440C0F00F40E0
:108A500000C0044000F10F409C02FF1F00C00C400A
:108A6000044B054AB3F87230C3F30321DBB25170F3
:108A7000137070479C02FF1F00C00C402DE9F04F9F
:108A8000974CDFF87CC2974EDFF878E29648DFF823
:108A90007882964B9649974F41F23C0541F2300956
:108AA000625942F00062625154F8092042F00062BB
:108AB00044F809200022CCF824204FF00D0ACCF80D
:108AC0002C204FF01009F2614FF0040CCEF8042076
:108AD000012604F5825EC0F808A0C8F808A0C0F816
:108AE0000C90C8F80C90C0F820C0C8F820C04262B2
:108AF000C8F824200660C8F80060DEF8009049F04D
:108B00000209CEF8009054F805A003F5845941F20B
:108B1000840E4AF0020A4FF0B60B44F805A00A7121
:108B200041F28C0581F804B041F29004C9F800705C
:108B300041F2940A41F2980923F80E606FF0030B9A
:108B400041F2880E43F805B00126185141F29E0506
:108B500023F80A2041F2960443F8092041F28600E6
:108B600041F29C0943F80E6003F5855E23F805C0C9
:108B7000614E23F804C041F2A4051A5241F2AC043C
:108B800023F8092041F2B0004FF0A8094A7141F2E0
:108B9000B40A81F80590CEF8006041F2B80941F2BC
:108BA000A80E564E5A531A5141F2BE051E500220CD
:108BB0006FF0070623F80A0041F2B60443F8096093
:108BC00043F80E0048F6040E23F805E041F2A6092A
:108BD00048F204051D5341F2BC0E40F2011423F883
:108BE000094040F2224923F80E90D3F80CE0434E9E
:108BF00003F5865967444EF0200E4FF0B80AC3F8CB
:108C00000CE008368A7141F2C40E81F806A0C9F85A
:108C1000007041F2CC0734464FF0010623F80E6095
:108C200041F2D00943F807B041F2D40E41F2D8071F
:108C300043F8098041F2C80A23F80E2041F2DE0908
:108C4000DA5141F2D60841F2C60E41F2DC070126A4
:108C50004FF0A90B43F80A6023F809C003F58756C3
:108C600023F808C041F2E40A23F80E2041F2EC098F
:108C7000DA5341F2F008CA7181F807B001F51A2100
:108C800041F2F40C41F2F80E41F2E8071031316084
:108C900041F2FE0B23F80A2041F2F60643F80920C0
:108CA00041F2E60143F8084041F2FC0A6FF0070484
:108CB00023F80C0048F6044943F80E4040F22262C3
:108CC000D85140F2011023F80B909D53585223F8CD
:108CD0000A20DA6842F08002DA6062B6BDE8F08FFE
:108CE0000070044000A0044000B003400080004039
:108CF000001002400800FF1F10B00340EC00FF1FEF
:108D000000B0044000C0044000B00B400249034AD8
:108D100001230B601360704700B0034000B00B40AC
:108D2000704700BF704700BF704700BF704700BF6B
:108D3000704700BF704700BF704700BF704700BF5B
:108D4000704700BF09490A4B4A6922F480124A6100
:108D50001A6D22F020021A651A6D42F002021A659D
:108D60001A6D42F001021A65704700BF40F00F40D3
:108D700000A0044009490A4B4A6922F480124A6162
:108D80001A6D22F020021A651A6D42F002021A656D
:108D90001A6D22F001021A65704700BF40F00F40C3
:108DA00000A00440094B0A4A596941F480115961F5
:108DB000116D21F002011165116D41F02001116565
:108DC0001A6822F480121A60704700BF40F00F400A
:108DD00000A00440024B1869C0F30050704700BF68
:108DE00040F00F400020704701280ED008D3022821
:108DF00004D1084B1869C0F3005070470020704739
:108E0000054B1869C0F3C0307047034B1869C0F3B5
:108E10000040704740F00F4080F00F40704700BFA7
:108E2000704700BF0020704705281CD8DFE800F01D
:108E3000070B0F1317030D4B588880B270470B4B6D
:108E4000988980B27047094B588980B27047074BA8
:108E5000188980B27047054B188880B27047034B61
:108E6000D88980B270470020704700BFEC00FF1F18
:108E700003281BD8DFE800F0140E08020C4A0D4B43
:108E8000927A33F812007047094A0A4B527A33F843
:108E900012007047064A074B127A33F812007047E7
:108EA000054A044B127C33F81200704700207047CB
:108EB0000800FF1F4803FF1FEC00FF1F032808D80E
:108EC000DFE800F0140E08020B4A0C4B927A23F8EC
:108ED00012107047084A094B527A23F81210704753
:108EE000054A064B127A23F812107047044A034BC6
:108EF000127C23F8121070470800FF1F4803FF1F61
:108F0000EC00FF1F0E490B690A6910B50C69920944
:108F1000C3F3002302F00202E408134304F0040444
:108F20001C4306D0072C04D0202000F0E5FF20468B
:108F300010BD0128F8D1202000F0D6FFF7E700BFD0
:108F400080F00F4038B50D4C0D4DB4F87410687AB0
:108F5000FFF7B4FFB4F87610A87AFFF7AFFFB4F8C4
:108F60007010287AFFF7AAFFB4F87230054AC3F3ED
:108F70000321DBB25170137038BD00BF9C02FF1F8C
:108F80000800FF1F00C00C40024B4FF480425A60A3
:108F9000704700BF00F00F40024B4FF480429A60D0
:108FA000704700BF00F00F40014B04225A60704729
:108FB00000F10F40014B04229A60704700F10F400E
:108FC000024B1868C0F38000704700BF00F10F40EB
:108FD000704700BF704700BF704700BF704700BFB9
:108FE000704700BF014B40225A607047C0F00F40ED
:108FF000014B40229A607047C0F00F40F0B541F23B
:109000003006354F354DBC59354BDFF804E144F09F
:109010001004BC514FF400742C664FF400566C667B
:10902000304DC3F800E01C465E601D602368DB0124
:10903000FCD50138072805D8DFE800F0363A3E4273
:109040004604324A264B284858602848244B284E6C
:1090500000274FF0806400EA81455F631E60C3F81B
:109060008040C3F8845082B14FF0846500EA8240AA
:10907000C3F89040C3F89400C3F8A050C3F8A410FC
:10908000C3F8B050C3F8B420F0BD4FF08460C3F80B
:109090009020C3F8A000C3F8A410C3F8B020F0BD1E
:1090A0000F4B14485860D0E70D4B13485860CCE77D
:1090B0000B4B12485860C8E7094B11485860C4E789
:1090C000074B10485860C0E7054B0F485860BCE795
:1090D000034B0E485860B8E70070044000D00440CD
:1090E00000400A400F0080508720FE070000FC1F50
:1090F0000F0080008720FE038720FEC78720FE63C5
:109100008720FE278720FE138720FE0F8720FE0181
:109110000F0080D0384AD2F88030C3F30363022BAB
:1091200066D0D2F89030C3F30363022B62D0D2F83A
:10913000A030C3F30363022B08D0D2F8B030C3F3DE
:109140000363022B01D00020704703231B0103F1AE
:10915000402202F52022D2F88010C1F303410170B1
:10916000D2F8801011F4801118BF01218170D2F85B
:10917000801011F4001133D14170D2F88410C1F382
:109180008A41416003F1402303F52023D3F888107E
:10919000090E0172D3F88810090C4172D3F88810B7
:1091A000090A8172D3F88810C172D3F88C10090EA5
:1091B0000173D3F88C10090C4173D3F88C10090A91
:1091C0008173D3F88C30C373D2F880309B024CBFCC
:1091D0004FF084634FF08063C2F880300120704705
:1091E00001214170D2F8841021F060414160C9E74B
:1091F0000023ABE70123A9E700400A401A4AD2F84E
:109200007031C3F303630C2B2CD010B4417819BB1D
:109210004468164B03EA8443C2F874318368124AE7
:109220001BBAC2F87831C3681BBAC2F87C318378A4
:10923000002914BF4FF042624FF040620BB142F47C
:1092400080120378084910BC1B0403F470231343F5
:109250000120C1F8703170474368C3F31103C2F8AD
:109260007431DBE70020704700400A400000FC1F1B
:1092700070B5254A254B2648264C41F2380641F266
:109280003C01955945F400759551555845F4805564
:109290005550555825F4802555505A6C42F40072AB
:1092A0005A641A6C42F400721A64DA6B42F4007267
:1092B000DA639A6B42F480729A634369012243F441
:1092C000804343612260236843F0004343F44063DA
:1092D0002360FFF759FE4FF06053E360E36843F00B
:1092E0002003E360E36843F48033E360E36A43F020
:1092F0008053E362236823F001032360236823F093
:109300000063236070BD00BF007004400090044003
:1093100000F00F4000C00240704700BF70B50C461F
:1093200016460546002833D001281ED1FFF752FE0D
:109330001B4BEEB144F000645C63DA6AD200FCD5EA
:10934000DA6A42F08052DA62DA6A12F0F00FFBD089
:109350009C6B1A6842F44062E4B21A60E5B1012DD8
:1093600001D1FFF735FE204670BD0E4B002EE1D136
:1093700044F000445C63DA6AC2F30332032AFAD889
:10938000DA6A12F0F00FFBD09C6BE4B2204670BD9D
:10939000FFF702FE034BCCE7FFF7F6FD204670BD5A
:1093A00000D0024000C00240012870B505460C46BE
:1093B00016463AD035D3022820D1FFF70FFE214BB5
:1093C000FEB144F000645C63DA6AD200FCD5DA6A6C
:1093D00042F08052DA62DA6A12F0F00FFBD09C6B36
:1093E0001A68012D42F44062A4B21A6025D020D33D
:1093F000022D01D1FFF7F0FD204670BD124B002E6B
:10940000DFD144F000445C63DA6AC2F30332032A1A
:10941000FAD8DA6A12F0F00FFBD09C6BA4B22046A7
:1094200070BDFFF7B9FD084BCAE7FFF7D3FD054B49
:10943000C6E7FFF7A9FD204670BDFFF7C9FD20462E
:1094400070BD00BF00D0024000C00240134AA8B166
:109450004FF000635363D36ADB00FCD5D36A0F4936
:1094600043F08053D362CB6A13F0F00FFBD0886BCC
:109470000B6843F4406380B20B6070474FF00043C9
:109480005363D36AC3F30333032BFAD8034AD36A73
:1094900013F0F00FFBD0906B80B2704700D0024009
:1094A000344B9842F0B438D0334B98423DD0334BD4
:1094B00098424FD0324B984254D0324B984219D0F8
:1094C000072A96BF304B4FF4165353F82230002929
:1094D000B8BF0F310911B1FBF3F1C1F30423C9B2D5
:1094E00003704170C37843F02C03C370F0BC2F208D
:1094F000FEF7C4BF254F264C41F228064FF44075B5
:10950000BB5943F48063BB51256600236566C37075
:1095100083708371C3724371D2E71C4D41F23404EE
:109520002B5943F480632B51CAE7A3F5103341F262
:10953000340641F238079C59154D44F400649C519F
:10954000DC594FF4407644F40054DC512E60002383
:109550006E60DCE70D4D41F234042B5943F4805327
:109560002B51ADE7094D41F234042B5943F400531C
:109570002B51A5E700A0064000B0064000C0064001
:1095800000D0064000A00E40B42701000070044047
:1095900000D00440024602490248FFF781BF00BFE5
:1095A00000D8B80500B006400A4A13685168013374
:1095B000202B08BF00238B420AD010B41168064C40
:1095C000114408721360E37843F08003E37010BC29
:1095D000704700BF0001FF1F00B006400B4B996AA7
:1095E000DA6A91420FD09A6A511C1A44996292F831
:1095F00030109A6A0170202A01D0012070470022A1
:109600009A62012070470020704700BF0001FF1FD1
:10961000044A137803F0FF0013B1002313700120F4
:10962000704700BF5403FF1F014B1865704700BF10
:109630000001FF1F684620F007018D4631B52A4919
:109640000C79E4B2A00615D5284AD36A906A013392
:10965000202B08BF0023834206D0D06ACD79111891
:10966000E8B281F83000D3622149224B052008601E
:10967000126D1A60620625D4230603D4BDE831407A
:10968000854670471B4B1D68002DF7D1174C22688B
:1096900063689A421ED0FFF787FC6368124A591C20
:1096A000234461601B7ADBB2D37163680E4A202BBE
:1096B00008BF6560D37843F04003D370BDE8314004
:1096C00085467047FFF776FC074AD37803F0BF035F
:1096D000D370D1E7044AD37803F07F03D370BDE899
:1096E00031408546704700BF00B006400001FF1FB3
:1096F0005803FF1F5C03FF1FF8B5244D244F69700A
:10970000002241F23C062A70BC59224B44F00074FE
:10971000BC5107245C650138C027842601241A60E7
:10972000C3F88470DA64586098609E65C3F880401E
:10973000D3F8803039B323F02003164C144EC4F80C
:109740008030D4F88020144B144F41F2380022F0BE
:1097500010020821C4F880202160325842F480624F
:1097600032504FF4C0614022196058205960C3F84C
:10977000A0209F61FEF782FE01232B70A068BDE848
:10978000F84006F099BF43F02003D6E75401FF1FCD
:10979000007004400090034000A004400001090054
:1097A000024A034B11801860704700BF6403FF1F1B
:1097B0006003FF1F014B1880704700BF6403FF1F49
:1097C000084B187820B1084B586880B2C0EB0040B5
:1097D000064B074A1B881268B0FBF2F000FB03F04F
:1097E00080B270475401FF1F009003406403FF1FC5
:1097F0006003FF1F034B187808B1034B586880B211
:10980000704700BF5401FF1F00900340014B588870
:10981000704700BF5401FF1F024B0022D8645A60FA
:10982000DA64704700900340014B1879704700BF1D
:109830005401FF1F014B00221A7170475401FF1F92
:10984000014B1870704700BF2000FF1F014B1878B4
:10985000704700BF2000FF1F014B9860704700BF9A
:109860005401FF1F014B9868704700BF5401FF1F50
:10987000014B187B704700BF5401FF1F024B0122B0
:1098800018611A73586970475401FF1F38B50C4CA2
:1098900025690122290C0220FFF786FDA9B20122C9
:1098A0000220FFF781FD074B05465988012202205F
:1098B000FFF77AFD002340EA05402373606138BD5D
:1098C0005401FF1F2000FF1F704700BF014B18838A
:1098D000704700BF5401FF1FF0B4114D114B41F20E
:1098E000380420272A59802642F400624FF4807100
:1098F0002A51C3F8A070C3F8A060C3F8A01030B913
:1099000059615920D961F0BC1962FEF7B7BD064A0A
:109910005A615920DA61F0BC1A62FEF7AFBD00BF90
:109920000070044000B0044000010B0008B5FFF7D0
:10993000E9FA0138C0B205289ABF024B33F910008A
:10994000002008BDD427010038B500F13B03762B79
:109950000B4C08D80020208042F6AA22094907F0C3
:1099600041F8208038BD2388074D01FB02F18003B8
:1099700095FBF1F190FBF1F0181A00B22080EBE7B3
:109980007401FF1F56D5FFFFE0930400014BB3F9AC
:10999000000070477401FF1F884210D0204B002246
:1099A00001381A80052808D8DFE800F033210327A2
:1099B0002D1A012932D0022916D0002070478B1EA3
:1099C000042BFAD801A252F823F000BFEF9900004F
:1099D000B3990000FB990000079A0000E19900008C
:1099E00002291BD00429E8D14FF0FF30704703292A
:1099F00014D00629F8D00020704706290ED005297A
:109A0000F2D000207047042908D00129ECD00020B2
:109A10007047052902D00329CFD1E5E7012070471F
:109A20007401FF1F014B5860704700BF7401FF1F96
:109A3000014B5868704700BF7401FF1FFEF732BE2C
:109A4000044B0548002207211A6058609A6019608B
:109A5000704700BF10E000E000770100014B0022DA
:109A60001A60704710E000E0014B1868704700BFB3
:109A70007C01FF1F684620F007018D460C490D4A06
:109A80000B6801B4106801330B6020B11368013B0F
:109A90001360136843B1084B1A6812B11A68013A8F
:109AA0001A6001BC85467047044B01221A70F2E728
:109AB0007C01FF1F5803FF1F5C03FF1F5403FF1FA0
:109AC000044B00221A619A611A629A621A639A63BD
:109AD000704700BF008003405D4AF8B541F23C0486
:109AE00041F2380115595B4B45F0807515511559F8
:109AF00045F480051551545844F4006454505458AA
:109B000044F4805454505A6D42F004025A650028BF
:109B100079D1D3F884205049504C42F0C002C3F8A8
:109B200084205A6D40F6C31542F061025A659D606B
:109B3000D864D3F88C2042F08002C3F88C209A6D50
:109B400042F002029A659A6D42F080029A650A8894
:109B50003F20024018665C669A66FFF7B1FF3D4BF6
:109B60003F49DA683F48404E404C42F00802DA6014
:109B70005A6942F008025A61DA6942F00802DA6171
:109B80005A6A42F008025A62DA6A42F00802DA625D
:109B90005A6B2A2742F008024FF400755A631F6778
:109BA000C3F89850DA6E42F04002DA665A6D42F01D
:109BB00002025A651D6840F20442002745F008057C
:109BC0001D6042608260C260026132617261CF607A
:109BD0000A6842F40A6242F0010240F6C3100A60C9
:109BE00048601F661A683E2042F040021A60FEF785
:109BF00045FC302384F83E334820FEF73FFC202309
:109C000084F84833F8BD5A6D1349144842F0610294
:109C10006FF49C6440F2E1455A659D60DC649A6D86
:109C200042F002029A659A6D3F2442F080029A65E2
:109C30001C665866088840F271226FF41C7120403F
:109C4000986619619A6119629A6219639A6386E744
:109C500000700440008003401400FF1F7373730002
:109C60000060034000B0044000C0044000E100E098
:109C7000014B3F221A6670470080034058B1064BE3
:109C80006FF41C7140F2712219619A6119629A6233
:109C900019639A63704713E700800340F0B444F2FD
:109CA000A8324DF6F00510FB02F310FB25F5EC1A77
:109CB0002B445A1082B04FEA640143D40029C0F209
:109CC000838002F51C521032521A44BF02F57F32D3
:109CD00002F2FF32002CBCBF04F57F3404F2FF34E3
:109CE0009214181EB8BF00F57F3002F2E24292B221
:109CF000B8BF00F2FF3002EBA444A2EBA040A4B234
:109D000080B20225624B1978012907D16149624F5F
:109D10000A8000264C8088803D701E705F49630871
:109D20005208400857425E4245424FF400748A612F
:109D30000F618B620E6288630D63C1F8984002B0B8
:109D4000F0BC704700291DDB002D5EDDC5F51C5100
:109D500010318A1844BF02F57F3202F2FF329214AA
:109D6000002BB8BF03F57F3302F2E24292B2B8BFD4
:109D700003F2FF33A2EBA34398B200EB65439CB21E
:109D80000325BFE702F51C521032521A44BF02F5F8
:109D90007F3202F2FF32002CBCBF04F57F3404F2A4
:109DA000FF349214002BB8BF03F57F3302F2E24276
:109DB00092B2B8BF03F2FF3302EBA444A2EBA34379
:109DC000A4B298B205259DE7002D41DD05F51C5292
:109DD0001032521A231E4FEAA242B8BF03F57F3356
:109DE00002F2E242B8BF03F2FF3392B2281EB8BFBC
:109DF00000F5FF3002EBA3439CB2B8BF00F2FF10A6
:109E0000A4EB604080B201257CE705F51C521032BE
:109E1000521A44BF02F57F3202F2FF329214231E1F
:109E2000B8BF03F57F3302F2E242B8BF03F2FF335B
:109E300092B2281EB8BF00F5FF3002EBA3439CB2DC
:109E4000B8BF00F2FF10A4EB604080B2042559E7D0
:109E5000C5F51C5110310A44002B4FEAA242B8BF8D
:109E600003F57F3302F2E242B8BF03F2FF3392B24E
:109E7000002DB8BF05F5FF35A2EBA343B8BF05F22F
:109E8000FF1598B200EB65439CB206253AE700BF88
:109E90008001FF1F6803FF1F2A00FF1F008003408F
:109EA000014B01221A7070478001FF1F014B33F8EC
:109EB000100070476803FF1F064A074B108851883F
:109EC00092880844104483FB0023A3EBE07080B227
:109ED000704700BF6803FF1F56555555014B187852
:109EE000704700BF2A00FF1F024A13681843106022
:109EF000704700BF8401FF1F024A136823EA000075
:109F0000106070478401FF1F044A136819B923EADF
:109F10000000106070471843106070478401FF1FF5
:109F2000034B1B68034214BF01200020704700BF91
:109F30008401FF1F024A136823F06D03136070470A
:109F40008401FF1F034B18681A6822F06D021A6023
:109F5000704700BF8401FF1F044B18681A6822F085
:109F60006D0200F06F001A60704700BF8401FF1F90
:109F70002DE9F041174F184D184E04463878FEF77A
:109F800053FF80463878FEF773FF294647F6FF7285
:109F9000A8EB000006F026FD07B23078FEF744FF7C
:109FA00080463078FEF764FF2946A8EB000047F6AC
:109FB000FF7206F017FD06B2B819294647F6FF7280
:109FC000404206F00FFD2780A08066802046BDE855
:109FD000F08100BF1100FF1F0180FFFF1200FF1F73
:109FE00038B5084C2078FEF71FFF05462078FEF7AD
:109FF0003FFF47F6FF72281A0021BDE8384006F0FF
:10A00000F1BC00BF1000FF1F002210B50321044661
:10A010001046FFF783F90022C4F307211046FFF72B
:10A020007DF90022E1B21046FFF778F900210846D9
:10A030000122BDE81040FFF771B900BF38B5012219
:10A0400004460D4600200621FFF768F9002210465D
:10A050000521FFF763F9002101220846FFF75EF9A9
:10A060008207F3D5002210460221FFF757F900229C
:10A070001046C4F30721FFF751F90022E1B2104660
:10A08000FFF74CF9294601220020FFF747F900228B
:10A0900010460521FFF742F9002108460122FFF78B
:10A0A0003DF9C307F3D438BDF8B51646002204467F
:10A0B0000D4610460321FFF731F90022C4F30721B2
:10A0C0001046FFF72BF90022E1B21046FFF726F900
:10A0D0007EB1013D771E00243A1B0021B2FA82F2C4
:10A0E00008465209FFF71AF90134A64205F8010F94
:10A0F000F2D1F8BD2DE9F04104460E46174606217F
:10A1000001220020FFF70AF9002210460521FFF77F
:10A1100005F9002108460122FFF700F98107F3D570
:10A12000002210460221FFF7F9F800221046C4F37E
:10A130000721FFF7F3F800221046E1B2FFF7EEF82F
:10A14000002F4AD0013E002507F1FF380AE0A8EBB6
:10A150000502B2FA82F252090020FFF7DFF801355A
:10A16000AF423AD0013414F03F0016F8011FEED18F
:10A170000122FFF7D3F8A845F1D9002210460521A6
:10A18000FFF7CCF8002108460122FFF7C7F810F0CE
:10A190000100F2D101220621FFF7C0F8002210468B
:10A1A0000521FFF7BBF8002101220846FFF7B6F8AA
:10A1B0008207F3D5002210460221FFF7AFF80022F4
:10A1C0001046C4F30721FFF7A9F800221046E1B2B8
:10A1D0000135FFF7A3F8AF42C4D100221046052194
:10A1E000FFF79CF8002108460122FFF797F8C30704
:10A1F000F3D4BDE8F08100BF38B50D46C0EBC00414
:10A2000004F500600978FFF719FF697804F601008A
:10A21000FFF714FFA97804F60200FFF70FFF297972
:10A2200004F60300FFF70AFF697904F60400FFF75C
:10A2300005FFA97904F60500FFF700FFE97904F6A8
:10A240000600BDE83840FFF7F9BE00BF002238B570
:10A250000C46C0EBC00503211046FFF75FF805F57B
:10A2600000650022C5F307211046FFF757F80022CA
:10A27000E9B21046FFF752F8002211461046FFF7E8
:10A280004DF80022114620701046FFF747F80022D3
:10A29000114660701046FFF741F800221146A07089
:10A2A0001046FFF73BF80022114620711046FFF7D9
:10A2B00035F80022114660711046FFF72FF8002193
:10A2C000A07101220846FFF729F8E07138BD00BFF0
:10A2D000F0B5002283B00D46C0EBC0040321104648
:10A2E000FFF71CF804F500640022C4F307211046B0
:10A2F000FFF714F80022E1B21046FFF70FF8002232
:10A3000011461046FFF70AF800221146064610468D
:10A31000FFF704F80022114604461046FEF7FEFF40
:10A320000022114607461046FEF7F8FF00221146AC
:10A330008DF804001046FEF7F1FF002211468DF85B
:10A3400005001046FEF7EAFF00218DF80600012205
:10A350000846FEF7E3FF8DF800608DF80140BDF878
:10A3600000202B888DF807009A4202D0002003B00D
:10A37000F0BDAB78BB42F9D16B680198C01AB0FA56
:10A3800080F04009F3E700BF38B54FF400650122C3
:10A3900006210020FEF7C2FF002210460521FEF72D
:10A3A000BDFF002101220846FEF7B8FF8207F3D562
:10A3B000002210460221FEF7B1FF00221046C5F32D
:10A3C0000721FEF7ABFF00221046E9B2FEF7A6FF19
:10A3D0000024A4F13F020021B2FA82F20846520999
:10A3E0000134FEF79BFF402CF3D1002210460521DB
:10A3F000FEF794FF002108460122FEF78FFFC307F6
:10A40000F3D44035B5F5804FC1D138BD70B50546A0
:10A4100040F2FF700C461646FFF7F6FDD32821D018
:10A42000002140F2FF70FFF709FEFFF7ADFF242285
:10A4300029460020FFF75EFE214640208022FFF7DC
:10A4400059FED32140F2FF70FFF7F8FD2946242280
:10A450000020FFF729FE214680224020BDE8704001
:10A46000FFF722BE002EDBD1F0E700BFF0B51D4C98
:10A470001D4FA569E369DFF874E003FB05F387FB73
:10A480000327421ADE17002AC6EB6736B8BF5242CE
:10A49000B242B8BF44F62063DEF80060B8BF534351
:10A4A000114A334482FB0362DF175213A2EB070CFD
:10A4B00044F6206606FB1C33CEF8003085B1884296
:10A4C00008DB0EDD2168BA1A494210448842B8BF41
:10A4D0000846F0BD216860448842A8BF0846F0BD28
:10A4E0000846F0BD9C02FF1FAD8BDB688801FF1F93
:10A4F0002DE9F84F5C4D95F825E02E68BEF1060F6A
:10A500000746884691461C4602D0BEF1000F73D123
:10A5100095F82900D7F800B0400807F017FA594617
:10A520008246584607F066FA504907F063FA01463A
:10A53000504607F05FFA8246A869C0EB0010C000E1
:10A5400007F004FA0146504607F008FB07F0A6FCA6
:10A55000A4EB09024C45B8BF7642002AB8BF52426C
:10A5600090424FEAE27371EB03034FF48040A8BFBF
:10A570000026FFF7D5FC012858D0304607F0E6F951
:10A580003C6880460146204607F0D2FBC8B1002E49
:10A5900038D1EB69A86903EB830203EB420300FBAC
:10A5A00003F007F0D3F9324907F0D8FA0146204604
:10A5B00007F018F904463860204607F0E1FBBDE8D3
:10A5C000F88F4146204607F0D1FB0028F4D00EB3A7
:10A5D000AB69E86900FB03F007F0B8F9254907F01B
:10A5E000BDFA0146204607F0FBF8044638602046D5
:10A5F00007F0C6FBBDE8F88FBEF1070F20D00020A2
:10A600000021A5E7AB69E86900FB03F007F09EF9BC
:10A610001849C9E7EB69A86903EB830203EB42031E
:10A6200000FB03F007F092F91149D8E7404607F024
:10A630008DF904463860204607F0A2FBBDE8F88F8C
:10A640000168084607F0D6F90B4907F087FA07F0CA
:10A6500025FCEB6BAA698E46A3FB000103FB0E11E0
:10A66000D31707F0B3FB73E79C02FF1F0000C04045
:10A670000050434800409C460000F042014B1878CF
:10A68000704700BF8C01FF1F014B1870704700BF5F
:10A690008C01FF1F38B50E4DAB6C1361401A0023BF
:10A6A0001446536110600B494FF6FF7206F09AF999
:10A6B0002369206003FB00F000282A68B8BFFF3040
:10A6C0000012A0615142BDE8384006F08BB900BFCE
:10A6D0009C02FF1F0100FFFF2DE9F84F394FD7F80B
:10A6E0004C803E6D5661C2F81080144697F82520C4
:10A6F000054699464AB9B8F10003B8BF0733002EA2
:10A70000B8BF03364FEAE308B610681A20602E4936
:10A710004FF6FF7206F066F9D4E902AB616920607A
:10A720001AEB000A4BEBE07BC4E902AB71B34FEAD2
:10A73000094292FBF6F25142504606F053F9236863
:10A74000824603FB08F34FEAE07B002BC4E902AB2F
:10A7500080FB06ABB8BFFF33BAF1000F4FEA2320EE
:10A760007BF100031EDB4FEA1A4343EA0B43184414
:10A77000A06197F82530082B0ED1002D08DDB86BAD
:10A78000BD6F000290FBF5F0BDE8F88F0A46D3E7F5
:10A7900010D12846BDE8F88F4A465142BDE8F84F2F
:10A7A00006F020B94FF6FF7200231AEB020A4BEBBA
:10A7B000030BD8E7B86BBD6F000290FBF5F0404289
:10A7C000BDE8F88F9C02FF1F0100FFFF2DE9F0415B
:10A7D00014460E461A46594206F004F9244A136BF1
:10A7E000516B2361002BB8BF0733DD10D4E902237E
:10A7F000801B00298846B8BF01F10308161843EBF7
:10A80000E077616120604FEAA808C4E9026739B3C4
:10A81000184A92FBF8F25142304606F0E3F82368FA
:10A8200003FB05F3002B06464FEAE07780FB0801A7
:10A83000B8BF03F2FF33002871F10002C4E90267D8
:10A840004FEAA3230EDB000C40EA01401844A0614C
:10A8500040F6C312084906F0C5F800B2BDE8F08121
:10A860000A46D9E74FF6FF76002780197941EAE7D3
:10A870009C02FF1F0000C3093DF6FFFFF8B5144618
:10A880000D461A46594206F0ADF8D4E902231F4E90
:10A8900000B2451B716B306B2061561943EBE577B5
:10A8A00025606161C4E9026739B3194A92FBF1F28C
:10A8B0005142304606F096F82269236803FB02F302
:10A8C0006269002B06464FEAE07780FB0201B8BFC1
:10A8D000FF33002871F10002C4E902674FEA232325
:10A8E0000DDB000C40EA01401844A06147F6FF72FE
:10A8F000084906F077F800B2F8BD0A46D9E74FF6E6
:10A90000FF76002780197941EBE700BF9C02FF1F0B
:10A910000000FF7F0180FFFF82B02DE9F04F1DB2E4
:10A920001C1487B005EBD57604EBD475B94CDDF873
:10A9300064E0139F01977610A680159E05966D1012
:10A94000169EE5800296179E04968146189E6068C2
:10A9500011930EEBDE770396DFF8CC82149D8A46C6
:10A96000934606F08FF8019B1E6898F82530A0608A
:10A9700006EBD676063B7F1046F34F06032B00F21C
:10A980002181DFE813F0B500F9005E00040000202B
:10A99000FEF7CCFF98F82820012A834600F070814A
:10A9A0005846FFF73FF8029B1B680293184607F0D2
:10A9B000E7F9D8F8142080EAE07EAEEBE07E964519
:10A9C00080F20C8198F82930D8F820609249934A97
:10A9D0000EFB03F006FB00F0000381FB0013C11720
:10A9E000C1EB6311236A194482FB01325211CB1768
:10A9F000D61A642000FB16102062002102980493EE
:10AA0000039207F0B3F9002800F01382039A049B25
:10AA1000E18BD8F838609B1A0B449BB203F5804158
:10AA2000E38309B23302F601D8F8782093FBF2F3FE
:10AA3000019A7B481360D8F8783096FBF3F636B26B
:10AA40006BE0029BD3F800B0584607F099F998F8EC
:10AA500029307149714A80EAE07EAEEBE07E03FB6B
:10AA60000EF0D8F8203003FB00F0000381FB001348
:10AA7000C117C1EB6311236A194482FB01325211E1
:10AA8000CB17D01A4FF0640E0EFB101E039000215E
:10AA90005846C4F820E00293019207F067F90028B5
:10AAA00000F0A980019A029BE18B9B1A0B449BB298
:10AAB00003F58041E38309B2594806F0D3F8C0F3A7
:10AAC0000F4328806B800120FEF730FF98F8283074
:10AAD000012B00F0DB80FEF7A5FFFEF771FEA0F56D
:10AAE000FF407F3800B2FEF7B7FE4FF0000B1CE0CE
:10AAF0000120FEF71BFF98F82E20012A834600F064
:10AB0000CA8098F82820012A7ED05846FEF78AFF8E
:10AB10000020FEF7A1FE4248594606F0A3F8C0F314
:10AB20000F4328806B804FF0000B3B464A46B5F937
:10AB300000103046FFF7A2FE3B46208252465846A0
:10AB4000B5F90210FFF79AFE237860827BBB238A57
:10AB5000A384344805F0BEFF324805F0E5FF2A889B
:10AB60006B88A06252005B002A806B8007B0BDE852
:10AB7000F04F02B0FFF792B8FEF768FE012855D0FB
:10AB8000FEF71EFE98F82C30A0F5FF407F38012B11
:10AB90000FFA80F800F047810020FEF743FF40469F
:10ABA000FEF75AFE41461E48A4F81E80B5E7A18C68
:10ABB0002182002200230021C9E902236182CAE91F
:10ABC0000223C6E70021164806F04CF84FF0000BB0
:10ABD000C0F30F4328806B805E46A6E759461048B5
:10ABE00006F040F8C0F30F42A4F81EB028806A8037
:10ABF0004FF0000B99E75846002107F099F800281C
:10AC000057D1B4F91E1057E70BF5FF437F330FFA06
:10AC100083FB7AE78C01FF1FF11976051F85EB5145
:10AC20009401FF1F9C01FF1F9C02FF1F4FF48060D7
:10AC3000FFF776F9012811D04FF40070FFF770F993
:10AC4000012801D1049B4BB94FF40060FFF768F96C
:10AC50000128B7D1019B1B68002BB3D098F82C308A
:10AC6000012B00F03C81C0F0FE80022B40F02C81D3
:10AC70006369032B3FF657AFDFE803F0A4452424B4
:10AC800000F5FF437F330FFA83FB89E600F5FF40B1
:10AC90007F3000B21FE798F82910D8F820200398D9
:10ACA0004908FEF751FEFEF771FE83440FFA8BFB55
:10ACB00027E7E38B039A1A4493B2A3F58041E38319
:10ACC00009B2F9E6584600262682668206F036F872
:10ACD000484606F033F8504606F030F805996269A8
:10ACE00000230B600299022A0B6000F0B4818020DF
:10ACF000FFF7FAF80020FEF795FEA069FEF7ACFD1D
:10AD0000B4F918105FE7D4F818B098F829308BEA36
:10AD1000EB715B08C3EB0342A1EBEB71914280F254
:10AD20009581D8F86010D8F82020CF4E01FB03F3AE
:10AD3000C2EBC23202FB03F3B8F8662086FB0316AF
:10AD4000B2F5007F4FEAE373C3EBA64600F09481AF
:10AD5000B2F5806F00F09081B2F5006F00F0AE8127
:10AD6000E368D8F83820C148D8F878104FEAC21BF9
:10AD70009BFBF1FB03FB0BFBA0FB0B3B0020FEF757
:10AD800051FEA069FEF768FDB4F91810B84805F047
:10AD900069FFB8F866302880B3F5007FC0F30F4034
:10ADA0004BF34F3B688000F07A81B3F5806F00F081
:10ADB000768198F8423013F0020332D102221E4607
:10ADC0006261B2E6E26842F210739A4200F23081A8
:10ADD000D8F83830A548D8F8781001324FEAC31BAC
:10ADE0009BFBF1FB02FB0BFBA0FB0B3B0020E2609B
:10ADF000FEF718FE0020FEF72FFD00219C4805F00D
:10AE000031FFB8F866302880B3F5007FC0F30F40FB
:10AE10004BF34F3B688000F03C81B3F5806F00F04E
:10AE20003881002681E61846FEF780FDFEF7FAFD20
:10AE3000B5E60298002106F07BFF20B90646B4F97A
:10AE40001E100346F0E5E28BD8F83800324492B287
:10AE5000C0EB0063A2F58041C0EB4060E28309B221
:10AE60001B02C601E0E5E36842F21072013393422F
:10AE7000E36000F2A180D8F838207C48B8F866106A
:10AE8000D8F878604FEAC21B9BFBF6FB03FB0BFB79
:10AE9000A0FB0B3BB1F5007F4BF34F3B00F08780ED
:10AEA000B1F5806F00F083800020FEF7BBFD00202D
:10AEB000FEF7D2FC00216E4805F0D4FEC0F30F432C
:10AEC00028806B80002630E60021694805F0CAFE24
:10AED0000026C0F30F4328806B80B34625E6184652
:10AEE0000393FEF70FF801460290207FFEF754FD12
:10AEF000039B029A019018462277FEF717FD98F8F7
:10AF00002820012A034604BF00F5FF437F3318467B
:10AF10000293FEF787FD019B002B029B76DB39D065
:10AF200003F515435433B8F93C1098F829205148DB
:10AF3000520803FB01F393FBF2F380FB0320184458
:10AF4000DB17C3EBE03080B2FEF766FCFEF738FC9F
:10AF500000230FFA80F8584623826382019305F09C
:10AF6000EDFE484605F0EAFE504605F0E7FE019B7F
:10AF70001846FEF765FC4FF40040FEF7B5FFA8F554
:10AF8000FF437F3B0FFA83F84046FEF765FC4146DE
:10AF90003748C2E50120FEF7C9FC98F82830012B9C
:10AFA00041D000F5FF437F330FFA83F8E7E7019ABA
:10AFB0004FEA4B03136077E700231846E360FEF780
:10AFC0002BFC98F82C302BBB98F8423043F001034F
:10AFD00088F8423058464FF0000BA4F810B0A4F89F
:10AFE00012B005F0ABFE484605F0A8FE504605F04D
:10AFF000A5FE059A00231360029A58461360FEF7D7
:10B000001FFC4FF40040FEF76FFF8EE503F5D543BC
:10B010002A3388E7022BDDD198F8423043F002034F
:10B0200088F84230D6E700F5FF437F3318B2B8E71F
:10B030000020FEF7F1FB98F84230012243F00203B2
:10B0400088F8423062614FF0000B6EE503236361C4
:10B050004FF0000B69E53046FEF7F2FB4FF400407D
:10B06000FEF742FF46E600BF851DD96F5917B7D1DD
:10B070009401FF1F01800080029B1B680293184609
:10B08000002106F073FE029B70B1ABEB0606A661D1
:10B0900066E6019A4FEA4B031360002645E5019AE4
:10B0A0004FEA4B03136084E61846002106F040FE89
:10B0B00000283FF455AE5E44A66151E6019B1B6833
:10B0C000002BE2DC3FF44CAEF5E700BF024B002260
:10B0D0005A61DA609A6170478C01FF1F014BB3F926
:10B0E0001E0070478C01FF1F08B5054B054918600D
:10B0F0000422FEF7D9FF044B01221A7008BD00BFDD
:10B100003408FF1F3808FF1FB801FF1F024A1368E9
:10B1100001331360704700BF3808FF1F2DE9F04B63
:10B120002D4B2E4D1E6ADA6D2D4C2E4F80EAE07E9F
:10B13000AEEBE07E85FB0E314FEAEE73C3EB2113DD
:10B140000EFB03F085FB0013C017C0EB231306FBB7
:10B1500003F3D4E9020187FB037E02EB8207DB17CE
:10B160006268C3EBEE0310EB030B02F101024FEA3E
:10B170008707B7FBF6F6A5FB063641F1000CB2EBEC
:10B18000561FC4E902BC626023DBD4F81080DFF8EC
:10B190005890676959F8286000234FF4C8725846E0
:10B1A000614606F063FE08F1010185FB0135CB170E
:10B1B000C3EB651500220023BE1BC4E902236423F0
:10B1C00003FB15150644002349F828006661256134
:10B1D0006360BDE8F08B00BF9C02FF1F1F85EB5131
:10B1E000B801FF1F676666663C08FF1F014B586980
:10B1F000704700BFB801FF1F014B1868704700BFC0
:10B200003808FF1F014B1860704700BF3808FF1F48
:10B21000054B1B78012B00D07047044B044918687C
:10B220000422FEF767BF00BFB801FF1F3408FF1FED
:10B230003808FF1F044B93F8643003B170474FF494
:10B240000030FEF759BE00BF9C02FF1F034B0449AC
:10B250001B68044A4B60052000F028BFD003FF1F85
:10B260002404FF1F1804FF1F094B9A7842B95B782A
:10B27000142B09D80749084A096842F82310704777
:10B28000064B04221A707047044B03221A70704751
:10B290002404FF1FD003FF1F7C03FF1F1804FF1FA0
:10B2A000034A044B12685A60092002F0DBBA00BF5F
:10B2B000D003FF1F2404FF1F054B06495A780120C5
:10B2C0008242087002D1044A5B681360704700BF75
:10B2D0002404FF1F0E04FF1F0404FF1F014B022262
:10B2E0001A7070470E04FF1FF0B4084F084E094D46
:10B2F000094C0A480A490B4A00233B7033602B6013
:10B30000237003600B601360F0BC70470E04FF1FD6
:10B310000404FF1F1004FF1F7403FF1FD003FF1F4F
:10B320002C04FF1F7803FF1F014B00221A70704787
:10B330000E04FF1F28494B78032B32D8DFE803F0B7
:10B3400026110602254B0A225A6070472449254BD4
:10B3500000220A6003F1280143F8042B8B42FBD141
:10B36000704770B41E4E306870B11E4A4D68136845
:10B37000AB421ED01146002303E051F8044FAC420B
:10B3800018D001338342F8D170BC7047144A136857
:10B39000092B0AD81348496840F823100133136079
:10B3A00070470E4B03221A7070470C4B09221A701B
:10B3B00070470023411E8B420BD200F180400138C0
:10B3C00002EB800002EB83035A6843F8042B8342AC
:10B3D000FAD13160D8E700BF2404FF1F1804FF1F13
:10B3E000F409FF1FCC09FF1F2B4A5378092B50D8B3
:10B3F000DFE803F010161C232A33393F450527499F
:10B4000053680B60264A002B3ED0136823F00803D4
:10B4100013607047214953680A6813440B60F1E7D1
:10B420001E4952680B689B1A0B60EBE71B49526878
:10B430000B6803FB02F30B60E4E7184952680B68E2
:10B4400093FBF2F30B60DDE714495268086890FB48
:10B45000F2F302FB13030B60D4E7104953680A6848
:10B4600013400B60CEE70D4953680A6813430B6025
:10B47000C8E70A4953680A6853400B60C2E7074AA5
:10B480001368DB431360BDE7136843F008031360E0
:10B490007047024B1B68B5E72404FF1FD003FF1F52
:10B4A0007803FF1F354B5B780A2B63D8DFE803F086
:10B4B000141B222A323C434A515806003049314A73
:10B4C000086813680B6010602F4A002B4DD013687A
:10B4D00023F0080313607047294A2A4B11681B6840
:10B4E0000B441360F0E7264A264B11681B68CB1A01
:10B4F0001360E9E7224A23491368096801FB03F353
:10B500001360E1E71E4A1F4B11681B6891FBF3F3C0
:10B510001360D9E71A4A1B491368096893FBF1F0D5
:10B5200001FB10331360CFE7154A164B11681B68F7
:10B530000B401360C8E7124A124B11681B680B439B
:10B540001360C1E70E4A0F4B11681B684B40136034
:10B55000BAE70C490A4B0A681B68D2430A60B3E792
:10B56000074B084A1B681360AEE7136843F00803F3
:10B5700013607047024B1B68A6E700BF2404FF1F3F
:10B58000D003FF1F2C04FF1F7803FF1F164B5B78AF
:10B59000052B09D8DFE803F0090F151B2103134A17
:10B5A000136823F4807313607047104A136803F024
:10B5B0000F03136070470D4A136823F010031360E4
:10B5C00070470A4A136823F0200313607047074A44
:10B5D000136823F0400313607047044A136823F094
:10B5E00080031360704700BF2404FF1F7803FF1F10
:10B5F000104A114B11685B68104A8B42136809DAD4
:10B6000023F0030343F00403136079B123F008032C
:10B61000136070470BBF23F0060323F0050343F0CC
:10B62000010343F0020313600029EFD143F0080344
:10B6300013607047D003FF1F2404FF1F7803FF1F10
:10B64000820709D4CB060BD50749084A4968084B3D
:10B65000116004221A707047064B08221A70704756
:10B66000044B0A221A7070472404FF1F7003FF1F47
:10B670000E04FF1F1804FF1F014B00221A707047B1
:10B680000E04FF1F104B5B78032B07D8DFE803F095
:10B69000190C07020D4A0E4B12685A6070470D4A8A
:10B6A0000B4B12685A6070470B4B1A680B48084BDB
:10B6B0000B49007809781A71120A5A71D871997178
:10B6C0007047084BF1E700BF2404FF1F2C04FF1F45
:10B6D0001804FF1FD003FF1F0404FF1F0E04FF1FE9
:10B6E0007403FF1F7003FF1F014B02221A70704783
:10B6F000D403FF1F024A034B52681A60704700BF11
:10B700002404FF1F0404FF1F284A53780C2B0CD875
:10B71000DFE803F0071E141923282E33383D424773
:10B720000C00234B1B68180704D47047204B1B6880
:10B73000DB05FAD51F4B52681A6070471C4B1B681B
:10B74000DB07F7D470471A4B1B68D807F2D5704750
:10B75000174B1B681907EDD57047154B1B68590728
:10B76000E8D47047124B1B6813F0050FE2D1704705
:10B770000F4B1B689B07DDD470470D4B1B68980768
:10B78000D8D170470A4B1B68D906D3D47047084BF1
:10B790001B689B06CED47047054B1B685806C9D45E
:10B7A0007047034B1B681906C4D470472404FF1F5D
:10B7B0007803FF1F0404FF1F084A1368072B0BD8E8
:10B7C00030B40749074C0D6844F8235030BC064894
:10B7D0000133406808601360704700BF1004FF1F0A
:10B7E0000404FF1FE403FF1F2404FF1FF0B5204BD8
:10B7F000204A5B68204D0124B3F5006F83B01470BC
:10B80000287001DC0C400AD01C4B0021DA1D03F823
:10B81000011B9342FBD12B782B7203B0F0BD18466D
:10B820006946FEF713FD9DF801309DF805009DF86F
:10B8300000209DF802E09DF807709DF80660AB704F
:10B840009DF80430A871EB716A70214685F803E019
:10B850002F716E71AB1C05F1080001E013F8012B8C
:10B860001144C9B283422972F8D103B0F0BD00BFC0
:10B870002404FF1FD403FF1FD803FF1FD903FF1F9A
:10B88000054A136833B1013B0448054950F82300C9
:10B8900013600860704700BF1004FF1FE403FF1F20
:10B8A0000404FF1F30B5134D6C7883B084B1012CB4
:10B8B00004D0114B03221A7003B030BDAB782A2B91
:10B8C000F7D1291D042240F2FB70FEF713FCF3E7C9
:10B8D00004220DEB020140F2FB70FEF7E5FB6A6803
:10B8E000019B9A42044B06BF01225A605C6003B080
:10B8F00030BD00BF2404FF1F1804FF1F014B0022AE
:10B900001A7070470E04FF1F70B5114E114D30684C
:10B91000114C2A786B686270B0F5006F636005D9CE
:10B920000E4A002107231170237070BD2946FEF7CF
:10B9300063FC29463068FEF7CBFC28B133686522EA
:10B9400001332270336070BD0723237070BD00BFC8
:10B950007003FF1F2404FF1F1804FF1F0E04FF1FA6
:10B9600070B52A4D2A4C2B786BB963685A1C2AD0C3
:10B9700003EB8303274A5B001360FEF775F8264A42
:10B98000012310602B7064787CB1012C0CD1FEF780
:10B99000D9FA10F4804630D11E4C2368DBB91F4A17
:10B9A0001368013B136070BD70BDFEF75DF81A4B64
:10B9B000184A1B681268C01A0028B8BF404290425B
:10B9C000EDD92C7070BD164B124A1B6803EB830334
:10B9D0005B001360D1E7FEF747F80F4B22681B6846
:10B9E000C31A002BB8BF5B429342D8D90D4A2E70C0
:10B9F000136843F01003136070BD0A4A13680021F6
:10BA000023F010032970136070BD00BF7403FF1F83
:10BA10002404FF1F3008FF1F0804FF1F0404FF1F3A
:10BA2000D003FF1F7803FF1F094B9A783AB95A7861
:10BA3000142A08D807495B6841F822307047064B42
:10BA400004221A707047044B03221A70704700BF1B
:10BA50002404FF1F7C03FF1F1804FF1F144B9A7858
:10BA60005AB95A78142A19D81249134B51F822207E
:10BA70005A60124A12783AB970470F4B04221A7072
:10BA80000E4A1278002AF7D00D4A5B6813600D4AFF
:10BA900043B1136823F0080313607047064B032279
:10BAA0001A70EDE7136843F008031360704700BF96
:10BAB0002404FF1F7C03FF1F1804FF1F0D04FF1F3A
:10BAC000D003FF1F7803FF1F0A4B9A783AB910B5CD
:10BAD0005C78142C07D9084B03221A7010BD064B52
:10BAE00004221A70704703F061FD044B43F82400F0
:10BAF00010BD00BF2404FF1F1804FF1F7C03FF1F9D
:10BB0000431E18B100BF13F1FF33FBD2704700BFD3
:10BB100041F238010D480E4A435830B443F4806373
:10BB20000C4C43504FF48075E560536908210B437A
:10BB3000536142F23413916000BF013BFCD1044ACF
:10BB4000536923F00803536130BC70470070044010
:10BB500040F00F4000A00440F8B5384D384C394F44
:10BB600000232B70FEF784F8FDF71CF941F2380131
:10BB700035486658354B364A46F400666650665876
:10BB800046F4805666504FF4807141608160C16018
:10BB9000016139617961596941F01E015961516949
:10BBA00041F030015161196821F0020119601968F2
:10BBB00021F008011960116821F010011160196865
:10BBC00041F004011960196841F01001196013680F
:10BBD00043F02003136042F2341300BF013BFCD159
:10BBE00041F2380116481B4C43581B4A43F480630A
:10BBF00043504FF48076E660536908210B4353614C
:10BC000042F23413916000BF013BFCD1124A5369E8
:10BC100023F00803536142F2341300BF013BFCD10F
:10BC20000A490D4A4B6923F004034B615369012112
:10BC300043F0080353612970F8BD00BFD001FF1F16
:10BC40000070044000C0044000B0044080F00F4089
:10BC5000C0F00F4000A0044040F00F40014B1878A6
:10BC6000704700BFD001FF1F064B074A1B691B0727
:10BC700003D4936801339360704753680133536072
:10BC8000704700BF40F00F40D001FF1F084909482E
:10BC90004B688A681A44A0FB020203EB830300206E
:10BCA0005B0052094860B3FBF2F38860CB607047D9
:10BCB000D001FF1F1F85EB51014BD868704700BFB3
:10BCC000D001FF1F0023194640FA03F212F0010FC2
:10BCD00003F1010318BF01310F2BF5D1CB0754BF7E
:10BCE00040F40040C0F30E00704700BF0023194627
:10BCF00040FA03F212F0010F03F1010318BF013102
:10BD00000F2BF5D181EAD03000F00100704700BF61
:10BD10001F4B2049F0B5002208251024DFF878E0F9
:10BD20009D6007462646104620254FF0010C47FA35
:10BD300002F3DB078E6040F252334CBFCEF8045062
:10BD4000CEF8085000BF013BFCD14C6040F2A91373
:10BD500000BF013BFCD10B695B0703D50CFA02F372
:10BD6000184380B240F2A91300BF013BFCD101325D
:10BD7000102ADCD10749084B8A6020229A6040F2E1
:10BD8000523300BF013BFCD1014B08225A60F0BD89
:10BD900040F00F4080F00F40C0F00F4038B5002455
:10BDA00085B22946234641FA03F212F0010F03F14E
:10BDB000010318BF01340F2BF5D1E30754BF45F43D
:10BDC0000045C5F30E052846FFF7A2FF42F23413E3
:10BDD00000BF013BFCD12846BDE83840FFF798BFC3
:10BDE0000220FFF7DBBF00BF0320FFF7D7BF00BF74
:10BDF0000420FFF7D3BF00BF70B520F48055ADB26B
:10BE0000002104460B4645F4006040FA03F212F0AC
:10BE1000010F03F1010318BF01310F2BF5D1C80742
:10BE200045BF46F6FF75254045F4084545F40065D5
:10BE30002846FFF76DFF6A4B00BF013BFCD124F49D
:10BE40000066B6B246F480501A4640FA02F111F08C
:10BE5000010F02F1010218BF01330F2AF5D1D907F2
:10BE600045BF47F2FF70204046F4104040F4805038
:10BE7000FFF74EFF0023194640FA03F212F0010FBC
:10BE800003F1010318BF01310F2BF5D1C0F3CF36F9
:10BE90004E40F643420406F0010648BF46F0020653
:10BEA00083040BD4684046F0040610F4FE6FB6B26B
:10BEB00002D046F00806B6B2304670BD2D0985EABC
:10BEC00010104006F5D1002EF6D142F2341300BF17
:10BED000013BFCD11A4644F4C05040FA02F111F083
:10BEE000010F02F1010218BF01330F2AF5D1D90762
:10BEF0004ABFC4F30E0044F4184040F4C050FFF7AA
:10BF000007FF00210B4640FA03F212F0010F03F184
:10BF1000010318BF01310F2BF5D181EAD03111F0A7
:10BF2000010F08BF1026420444BF46F02006B6B2F7
:10BF300083040BD485EA101546F040066906B6B2B4
:10BF4000BAD046F08006B6B2304670BD85EA101011
:10BF50004206F6D1002EAFD142F2341300BF013BAE
:10BF6000FCD124F4C0501A4680B240FA02F111F01C
:10BF7000010F02F1010218BF01330F2AF5D1DB07CF
:10BF80004ABF46F2FF7040F400402040FFF7C0FE79
:10BF900000210B4640FA03F212F0010F03F10103F6
:10BFA00018BF01310F2BF5D181EAD03111F0010F0B
:10BFB00008BF4FF48076410444BF46F40076B6B221
:10BFC000820458BF46F4806685EA101558BFB6B2A1
:10BFD0006B061CBF46F40066B6B2304670BD00BFAB
:10BFE0001C7E06004FF6FA73034043F00200FFF791
:10BFF00003BF00BF4FF6FB73034043F00300FFF79E
:10C00000FBBE00BF4FF6FC73034043F00400FFF794
:10C01000F3BE00BF1A481B49F8B50022DFF888E0DC
:10C02000194F1A4E1A4D1B4C1B4B02604FF4807077
:10C0300008808EF800203A6032602A60227003F592
:10C04000806143F8042F8B42FBD1144FFB7D73B901
:10C05000134E40F21A7440F2FA75A4F21A710422D7
:10C06000204631441444FEF71FF8AC42F5D17B7DE5
:10C0700013B90C4A1370F8BD0A4B01221A70F8BDAF
:10C080000404FF1FFC11FF1FD003FF1F2C04FF1F20
:10C090007803FF1F7403FF1F2C04FF1F2003FF1FE3
:10C0A0003004FF1F0E04FF1FF909FF1F30B58B7806
:10C0B00083B00446002B40F005814B78FE2B00F244
:10C0C000E886DFE813F01601B805AB05A1058D057C
:10C0D000E6065C044804E6063404200447053305FC
:10C0E0002905E606E606E606E606E606E606150580
:10C0F000BB03E606E606E606A70331069E031B061B
:10C100001306E6062906E606E606E606E606E6065F
:10C11000E606E606E606E606E606E606E606E606BF
:10C12000E606E606E606E606E6066805FC05F00510
:10C130000806E503DC05CF05EA05B7044303380329
:10C14000E606E606E606E606E606E606E606E6068F
:10C15000E606E606E606E606E606E606E606E6067F
:10C16000E606E606E606E606E606E606E606E6066F
:10C17000E606E606E606E606E606E606E606E6065F
:10C18000E606E606E606E606E606E606E606E6064F
:10C19000E606E606E606E606E606E606E606E6063F
:10C1A000E606E606E606E606E606E606E606E6062F
:10C1B000E606E606E606E606E606E606E606E6061F
:10C1C000E606E606E606E606E606E606E606E6060F
:10C1D00024031003E606E606E606E606E606E6069D
:10C1E000E606E606E606E606E6066306E606E60672
:10C1F000E606830545060B05E606E6067605170402
:10C20000E606E6060304E606EF03E606FE04E60697
:10C21000EA04D604E606E606E606E606E606C204F4
:10C220008A03E606760362034E0398068406E60652
:10C23000E606E606E606E606E606E606E606E6069E
:10C24000E606B8065B05CF067706D903CD03AB0437
:10C250009F04AB069304DC06C505C5060703E60686
:10C26000C102E606E6068902E7028002DD01D4018A
:10C27000E606DE02CC0126021A02FB020E02E606E8
:10C28000E606E606E606E606E6067501E6066D0142
:10C29000D5025A01E606E606E6066C025802E606F4
:10C2A00044023002B801E606A401E606E606900163
:10C2B000E606E606E606E6067D01FA014701E60126
:10C2C0003401210104231370062C0BD1CC4B1B78B5
:10C2D00043B15368CB4A1360CB4A2BB1136823F0A8
:10C2E0000803136003B030BD136843F00803136004
:10C2F000F8E7052C00F02A87062CF3D1019202F012
:10C30000DBFF019A5060E1E7052C00F0AD87062CB9
:10C3100001F06280072C01F0C181082CE2D1BB49F9
:10C320000122682003B0BDE83040FDF7BDBE052CFA
:10C3300000F00586062C01F0BC80072C01F09E81E0
:10C34000082CCFD1B2490122692003B0BDE83040AA
:10C35000FDF7AABE052C00F0AB87062C01F020806B
:10C36000072C01F0D381082CBCD1AA4901226D20F1
:10C3700003B0BDE83040FDF797BE052C00F05686AF
:10C38000062C01F0B280072C01F06881082CA9D19D
:10C39000A1490422882003B0BDE83040FDF784BEE7
:10C3A000062C9FD1019203F059FD019A50608DE750
:10C3B000062C97D1019203F03DFA019A506085E76F
:10C3C000052C00F06187062C01F02280072C01F07B
:10C3D0004D81082C86D1914901226C2003B0BDE823
:10C3E0003040FDF761BE052C00F03487062C00F0CC
:10C3F000EC87072C01F0BA80082C7FF473AF8849D2
:10C4000002226A2003B0BDE83040FDF74DBE052C86
:10C4100000F0E285062C01F08480072C01F0AE804C
:10C42000082C7FF45FAF7F490422A02003B0BDE851
:10C430003040FDF739BE052C00F04A87062C00F08D
:10C44000BD87072C01F00281082C7FF44BAF7649A1
:10C450000222AE2003B0BDE83040FDF725BE052C1A
:10C460007FF432AF03B0BDE83040FFF751BB062C7C
:10C470007FF438AF0192FEF731FE019A506025E754
:10C48000062C7FF42FAF0192FDF7ECF9019A506072
:10C490001CE7052C00F0EE86062C00F0B287072C76
:10C4A00001F0F480082C7FF41DAF604901226E205A
:10C4B00003B0BDE83040FDF7F7BD052C00F0A286C3
:10C4C000062C00F0BA87072C01F01081082C7FF4AD
:10C4D00009AF574904227C2003B0BDE83040FDF786
:10C4E000E3BD052C00F03485062C7FF4FBAE0192F1
:10C4F000FFF77EFC019A5060E8E6052C00F03085DD
:10C50000062C7FF4EFAE0192FFF76AFC019A5060AF
:10C51000DCE6052C7FF4D8AE03F096FC03B0BDE852
:10C520003040FFF719BB052C00F0B886062C00F050
:10C530003087072C01F0BA80082C7FF4D3AE3D4938
:10C540000222AC2003B0BDE83040FDF7ADBD052CA4
:10C5500000F07686062C00F04D87072C01F0AE80A7
:10C56000082C7FF4BFAE34490122AA2003B0BDE8F5
:10C570003040FDF799BD052C00F0FA84062C00F040
:10C580009F87072C01F0A280082C7FF4ABAE2B49CB
:10C590000422902003B0BDE83040FDF785BD052C96
:10C5A00000F08C86062C00F00287072C01F0068034
:10C5B000082C7FF497AE224904228C2003B0BDE8FA
:10C5C0003040FDF771BD062C7FF48CAE0192FDF773
:10C5D0002FFA019A506079E6052C00F02786062C88
:10C5E00000F00187072C01F02980082C7FF47AAE37
:10C5F00014490422B82003B0BDE83040FDF754BD13
:10C600000D04FF1FD003FF1F7803FF1FC402FF1F8D
:10C61000C502FF1FC902FF1FE402FF1FC802FF1F60
:10C62000C602FF1FFC02FF1F0A03FF1FCA02FF1FF3
:10C63000D802FF1F0803FF1F0603FF1FEC02FF1FA6
:10C64000E802FF1F1403FF1F052C00F04B86062C89
:10C6500000F09186072C01F06180082C7FF442AE37
:10C66000D1490122A92003B0BDE83040FDF71CBD2F
:10C67000062C7FF437AE019203F0F6FB019A50606E
:10C6800024E6062C7FF42EAE0192FFF715FB019AEB
:10C6900050601BE6052C00F02F86062C00F07286F9
:10C6A000072C01F02B80082C7FF41CAEBF4904221C
:10C6B000BC2003B0BDE83040FDF7F6BC052C00F00F
:10C6C0002B85062C7FF40EAE0192FFF78DFB019AAD
:10C6D0005060FBE5062C7FF405AE019203F0DCFB15
:10C6E000019A5060F2E5052C00F04B85062C00F015
:10C6F0000D86072C00F06A87082C7FF4F3ADAC4957
:10C700000422602003B0BDE83040FDF7CDBC052C0D
:10C7100000F08285062C00F09786072C00F07E87BB
:10C72000082C7FF4DFADA34904225C2003B0BDE8F0
:10C730003040FDF7B9BC062C7FF4D4AD0220019245
:10C7400002F000FB9C4B019A5860BFE5062C7FF479
:10C75000C9AD0120019202F0F5FA974B019A586099
:10C76000B4E5052C00F0AA84062C00F0F485072C13
:10C7700000F05C87082C7FF4B5AD90490422782046
:10C7800003B0BDE83040FDF78FBC052C00F02685D6
:10C79000062C00F04486072C00F0E887082C7FF474
:10C7A000A1AD87490222B22003B0BDE83040FDF7B9
:10C7B0007BBC052C00F01C85062C00F03786072C6E
:10C7C00000F0DC87082C7FF48DAD7E490222B0207A
:10C7D00003B0BDE83040FDF767BC052C00F0E983ED
:10C7E000062C00F04A86072C00F0A887082C7FF45E
:10C7F00079AD75490422742003B0BDE83040FDF7DF
:10C8000053BC062C7FF46EAD0192FEF7EFFC019A4B
:10C8100050605BE5052C00F0D784062C00F02686DE
:10C82000072C00F09B86082C7FF45CAD674904223E
:10C830009C2003B0BDE83040FDF736BC644D95F850
:10C840002F30990740F1568301200192FCF7CCFA72
:10C850000128019A00F05B81574B0021596033E5B4
:10C86000052C00F0D383062C7FF43CAD019203F03D
:10C87000CFFE019A506029E5052C00F07C84062C3F
:10C880007FF430AD019203F0BDFE019A50601DE5CA
:10C89000062C7FF427AD0192FDF720FB464B019A51
:10C8A000586013E5052C00F0AB83062C00F047869A
:10C8B000072C00F03383082C7FF414AD4549012286
:10C8C000942003B0BDE83040FDF7EEBB052C00F02E
:10C8D000B783062C00F01086072C00F03787082C51
:10C8E0007FF400AD3C490122652003B0BDE8304033
:10C8F000FDF7DABB062C7FF4F5AC0192FDF722FBC5
:10C90000019A5060E2E4052C00F03B83062C00F015
:10C91000DE85072C00F0E286082C7FF4E3AC2F497B
:10C9200004224C2003B0BDE83040FDF7BDBB052C10
:10C9300000F0A083062C00F0ED85072C00F0268681
:10C94000082C7FF4CFAC26490422502003B0BDE868
:10C950003040FDF7A9BB052C00F05E83062C00F0EB
:10C96000BD85072C00F01A86082C7FF4BBAC1D494E
:10C970000422482003B0BDE83040FDF795BB052CEC
:10C9800000F01884062C00F06685072C00F026863F
:10C99000082C7FF4A7AC14490422442003B0BDE85E
:10C9A0003040FDF781BB00BF0503FF1F1803FF1FC9
:10C9B000BC02FF1FB802FF1F1804FF1FD402FF1F95
:10C9C0000E03FF1F0C03FF1FD002FF1FF802FF1F03
:10C9D0009C02FF1FF002FF1FC102FF1FA802FF1FE2
:10C9E000AC02FF1FA402FF1FA002FF1F052C00F0D6
:10C9F0004B83062C7FF476AC019203F021FE019A62
:10CA0000506063E4052C00F05383062C7FF46AAC7D
:10CA1000019203F009FE019A506057E4052C00F0E2
:10CA20009B83062C7FF45EAC019203F0F7FD019A24
:10CA300050604BE4062C7FF455AC0020019202F0CC
:10CA400081F9C84B019A586040E4052C00F06E82D1
:10CA5000062C00F02785072C00F09886082C7FF420
:10CA600041ACC1490422702003B0BDE83040FDF75D
:10CA70001BBB052C00F01A82062C00F04982072C03
:10CA800000F09486082C7FF42DACB84901226F2069
:10CA900003B0BDE83040FDF707BB052C00F0A682CF
:10CAA000062C00F04585072C00F08085082C7FF4CB
:10CAB00019ACAF490222802003B0BDE83040FDF739
:10CAC000F3BA052C00F0C682062C7FF4F1AE019279
:10CAD00003F074FC019A5060FFF7F8BB062C7FF45A
:10CAE00001AC019202F0FCFB019A5060FFF7EEBB33
:10CAF000A04D95F82F3013F0010000F0EE810020DA
:10CB00000192FCF771F90128019A7FF4A5AE954BCB
:10CB100001215960FFF7D8BB062C7FF4E3AB0192EB
:10CB200002F0D0FB019A5060FFF7D0BB052C00F05B
:10CB30004982062C00F0A884072C00F02F86082CD0
:10CB40007FF4D0AB8C490422542003B0BDE83040C0
:10CB5000FDF7AABA052C00F0CF82062C00F0F48372
:10CB6000072C00F0E385082C7FF4BCAB834904223A
:10CB7000582003B0BDE83040FDF796BA052C00F010
:10CB80001282062C7FF4AEAB019203F029FD019ACC
:10CB90005060FFF79BBB062C7FF4A4AB0192FDF71E
:10CBA0007FF90020FDF782F96E4B019A5860FFF77C
:10CBB0008DBB052C00F08C82062C7FF493AB019288
:10CBC00002F050FB019A5060FFF780BB062C7FF407
:10CBD00089AB019202F0E8FD019A5060FFF776BB45
:10CBE000052C00F0D781062C00F05584072C00F0AE
:10CBF000B585082C7FF476AB5E490422402003B053
:10CC0000BDE83040FDF750BA062C7FF46BAB0192C3
:10CC100002F0C4FD019A5060FFF758BB052C00F0EC
:10CC2000A182062C7FF45EAB019202F0C5FC019A52
:10CC30005060FFF74BBB052C00F07C82062C7FF484
:10CC400051AB019202F0B2FC019A5060FFF73EBB7B
:10CC5000062C7FF447AB019203F012F9019A506061
:10CC6000FFF734BB062C7FF43DAB454B019218789F
:10CC7000FCF7DAF83B4B019A5860FFF727BB052C0D
:10CC800000F00B81062C7FF42DAB0192FDF7F6FC32
:10CC9000344B019A5860FFF719BB062C7FF422AB86
:10CCA0000192384BE3E7062C7FF41CAB0220019283
:10CCB000FDF7FCF82B4B019A5860FFF707BB062CD9
:10CCC0007FF410AB01200192FDF7F0F8254B019A9B
:10CCD0005860FFF7FBBA062C7FF404AB0192FDF716
:10CCE000EBF8204B019A5860FFF7F0BA052C7FF45F
:10CCF000EBAA03B0BDE83040FEF79CBA052C00F06B
:10CD00005382062C00F01283072C7FF4EBAA03B0A9
:10CD1000BDE83040FEF77CBA052C7FF4D5AA03B0FD
:10CD2000BDE8304002F006BD052C00F09981062CCC
:10CD300000F0E983072C00F00984082C7FF4D2AAC4
:10CD400011490422982003B0BDE83040FDF7ACB98A
:10CD5000062C7FF4C7AA019202F0BCFA019A506037
:10CD6000FFF7B4BA1804FF1FCC02FF1FCB02FF1F4E
:10CD7000DC02FF1F9C02FF1FB002FF1FB402FF1F57
:10CD80001100FF1F1200FF1FF402FF1F052C00F00F
:10CD9000A981062C00F0D182072C00F03784082CE2
:10CDA0007FF4A0AABB490122642003B0BDE8304053
:10CDB000FDF77AB9052C00F0EE81062C7FF492AADB
:10CDC000019203F019FC019A5060FFF77FBA052C1D
:10CDD00000F0E781062C00F0A082072C00F00E8402
:10CDE000082C7FF47FAAAC490222B62003B0BDE82C
:10CDF0003040FDF759B9052C61D0062C00F0B28205
:10CE0000072C00F0F383082C7FF46CAAA3490222BC
:10CE1000B42003B0BDE83040FDF746B9052C00F062
:10CE20007581062C7FF45EAA019203F003FC019A3F
:10CE30005060FFF74BBA052C00F07681062C7FF48A
:10CE400051AA019203F0C6FB019A5060FFF73EBA67
:10CE5000062C7FF447AA019203F018F8019A50605B
:10CE6000FFF734BA052C00F06B81062C7FF43AAA48
:10CE7000019203F0BBFB019A5060FFF727BA062C22
:10CE80007FF430AA019202F0F5FF019A5060FFF79B
:10CE90001DBA03231370FFF717BA4868012840F240
:10CEA0008D847F4B04221A70FFF71CBA4B68032B4A
:10CEB0000FD87C4B0A7983F82F20FFF713BA7A4BEF
:10CEC00001924968187803F039FB019A00287FF431
:10CED00009AA04231370FFF705BA0192FBF784FF38
:10CEE000019A00283FF413AE95F82F30D8073FF58C
:10CEF00006AEB1E401200192FBF776FF019A00280B
:10CF00003FF405AE95F82F309B077FF5A5AC9BE469
:10CF1000644B93F82F305360FFF7D8B9634901226F
:10CF2000942003B0BDE83040FDF7E4B848680192B2
:10CF300003F0FCF8019A0028CBD0FFF7D3B948687A
:10CF4000019202F0DDFF019A0028C2D0FFF7CAB9B2
:10CF500088880192FFF756F8019A5060FFF7C2B92E
:10CF600088880192FFF73EF8019A5060FFF7BAB93E
:10CF70004868019203F084F9019A0028A9D0FFF7CC
:10CF8000B1B94868019203F0DDF9019A0028A0D0F8
:10CF9000FFF7A8B94868019203F000F9019A002848
:10CFA00097D0FFF79FB9486803B0BDE8304003F061
:10CFB00053BB4868019203F0CBF8019A002888D04F
:10CFC000FFF790B94868019203F0D4F8019A00285D
:10CFD0003FF47FAFFFF786B94868019203F03AF853
:10CFE000019A00283FF475AFFFF77CB948680192B9
:10CFF00002F0F0FF019A00283FF46BAFFFF772B91F
:10D00000486803B0BDE8304003F0B0B9486803B0E9
:10D01000BDE8304003F038BB4868019203F07EF968
:10D02000019A00283FF455AFFFF75CB948680192B8
:10D0300003F062F9019A00283FF44BAFFFF752B9B1
:10D040004868019203F032F8019A00283FF441AF9A
:10D05000FFF748B9486803B0BDE8304003F09EB917
:10D060004868019203F000FA019A00283FF431AFBA
:10D07000FFF738B94868019203F0A4F8019A002834
:10D080003FF427AFFFF72EB9486803B0BDE8304042
:10D0900003F012BBC002FF1F1203FF1F1003FF1F8C
:10D0A0001804FF1F9C02FF1F1100FF1FF002FF1F4B
:10D0B000486803B0BDE8304003F0F2BA4868019216
:10D0C00002F00AFF019A00283FF403AFFFF70AB904
:10D0D0004868019202F0E4F8019A00283FF4F9AEA2
:10D0E000FFF700B94868019203F0DCF8019A0028C4
:10D0F0003FF4EFAEFFF7F6B84868019203F0E8F8A6
:10D10000019A00283FF4E5AEFFF7ECB8486803B099
:10D11000BDE8304003F0CABA88880192FEF76AFF82
:10D12000019A5060FFF7DEB8486803B0BDE83040B0
:10D1300003F08CBA486803B0BDE8304002F01EBB73
:10D14000486803B0BDE8304003F08CBA486803B0CB
:10D15000BDE8304002F04EB8486803B0BDE830404A
:10D1600003F098BA4868019202F016F8019A002874
:10D170007FF4B8A8ADE6486803B0BDE8304003F0DE
:10D180007DBA4868019202F0BFFF019A00283FF47F
:10D19000A0AEFFF7A7B8486803B0BDE8304003F081
:10D1A00067BA0192AF4B8CE6486803B0BDE83040E7
:10D1B000FEF728B84868019202F07AFE019A00282A
:10D1C0003FF487AEFFF78EB84868019203F038F954
:10D1D000019A00283FF47DAEFFF784B848680192B9
:10D1E00003F08AF9019A00283FF473AEFFF77AB88A
:10D1F0004868019203F062F9019A00283FF469AE91
:10D20000FFF770B84868019202F0CAFE019A002840
:10D210003FF45FAEFFF766B84868019202F0E6FFA0
:10D22000019A00283FF455AEFFF75CB848680192B8
:10D2300003F078F9019A00283FF44BAEFFF752B89B
:10D240004868019203F0C2F8019A00283FF441AE09
:10D25000FFF748B84868019202F014FF019A0028CD
:10D260003FF437AEFFF73EB8486803B0BDE8304042
:10D2700002F070BE4868019202F080FE019A002818
:10D280003FF427AEFFF72EB84868019202F0D0FEB7
:10D29000019A00283FF41DAEFFF724B848680192B8
:10D2A00003F0A6F8019A00283FF413AEFFF71AB86E
:10D2B000486803B0BDE8304002F0A0BE4868019263
:10D2C00002F0CCFF019A00283FF403AEFFF70AB842
:10D2D0004868019203F0A2F8019A00283FF4F9ADE2
:10D2E000FFF700B84868019203F0D2F8019A0028CD
:10D2F0003FF4EFADFEF7F6BF4868019203F05EF928
:10D30000019A00283FF4E5ADFEF7ECBF019202F070
:10D3100007FF019A5060FEF7D9BF524B019218786F
:10D3200003F034F9019A5060FEF7D0BF0192FDF787
:10D3300063FF019A5060FEF7C9BF019202F0BEFF81
:10D34000019A5060FEF7C2BF019202F0CFFF019A2E
:10D350005060FEF7BBBF019202F0B8FD019A506029
:10D36000FEF7B4BF404B0192187803F00FF9019A11
:10D370005060FEF7ABBF019203F096F8019A50603F
:10D38000FEF7A4BF019203F01FF9019A5060FEF767
:10D390009DBF019203F03CF8019A5060FEF796BFE2
:10D3A000019202F03BFE019A5060FEF78FBF01929E
:10D3B00002F060FF019A5060FEF788BF019203F00F
:10D3C00039F8019A5060FEF781BF019202F068FEC1
:10D3D000019A5060FEF77ABF019202F0C5FD019AF2
:10D3E0005060FEF773BF019203F0A2F8019A5060FB
:10D3F000FEF76CBF019202F0F5FF019A5060FEF754
:10D4000065BF019202F0C6FD019A5060FEF75EBF53
:10D41000019202F019FE019A5060FEF757BF019287
:10D4200003F07AF8019A5060FEF750BF019203F0C2
:10D430005DF8019A5060FEF749BF019202F0C4FD09
:10D44000019A5060FEF742BF019202F001FF019A7B
:10D450005060FEF73BBF019202F024FD019A50603C
:10D46000FEF734BF1200FF1F1100FF1F019202F0F0
:10D47000F5FF019A5060FEF729BF019202F074FE99
:10D48000019A5060FEF722BF019202F081FE019ADC
:10D490005060FEF71BBF019202F08EFE019A5060B1
:10D4A000FEF714BF019202F04DFE019A5060FEF7A4
:10D4B0000DBF019202F01EFD019A5060FEF706BFFB
:10D4C000019202F0E9FE019A5060FEF7FFBE019260
:10D4D00002F046FF019A5060FEF7F8BE019202F09A
:10D4E0002BFF019A5060FEF7F1BE019202F010FF8F
:10D4F000019A5060FEF7EABE019202F0E9FD019A3E
:10D500005060FEF7E3BE019202F0BCFF019A50604A
:10D51000FEF7DCBE019202F063FE019A5060FEF756
:10D52000D5BE019202F0A8FD019A5060FEF7CEBE72
:10D53000019202F05DFD019A5060FEF7C7BE0192B4
:10D5400002F024FF019A5060FEF7C0BE9E490422FB
:10D55000982003B0BDE83040FCF7CCBD9B490422C5
:10D560009C2003B0BDE83040FCF7C4BD98490222BE
:10D570006A2003B0BDE83040FCF7BCBD95490422E9
:10D58000A02003B0BDE83040FCF7B4BD92490422AE
:10D59000502003B0BDE83040FCF7ACBD8F490422F9
:10D5A000482003B0BDE83040FCF7A4BD8C490222FE
:10D5B000802003B0BDE83040FCF79CBD89490422BF
:10D5C0008C2003B0BDE83040FCF794BD86490422AE
:10D5D000602003B0BDE83040FCF78CBD83490422D5
:10D5E000442003B0BDE83040FCF784BD80490222EE
:10D5F000B42003B0BDE83040FCF77CBD7D49022279
:10D60000B62003B0BDE83040FCF774BD7A49012272
:10D61000642003B0BDE83040FCF76CBD77490422BC
:10D620005C2003B0BDE83040FCF764BD74490422BF
:10D63000782003B0BDE83040FCF75CBD714904229E
:10D64000B82003B0BDE83040FCF754BD6E4902225B
:10D65000AE2003B0BDE83040FCF74CBD6B4904225E
:10D66000882003B0BDE83040FCF744BD6849012282
:10D670006C2003B0BDE83040FCF73CBD6549012299
:10D68000692003B0BDE83040FCF734BD6249012297
:10D690006E2003B0BDE83040FCF72CBD5F4901228D
:10D6A000682003B0BDE83040FCF724BD5C4902228D
:10D6B000AC2003B0BDE83040FCF71CBD5949012245
:10D6C000AA2003B0BDE83040FCF714BD564904223F
:10D6D000902003B0BDE83040FCF70CBD5349042254
:10D6E0004C2003B0BDE83040FCF704BD5049042293
:10D6F0007C2003B0BDE83040FCF7FCBC4D4904225F
:10D70000BC2003B0BDE83040FCF7F4BC4A4901221C
:10D710006D2003B0BDE83040FCF7ECBC4749012266
:10D72000A92003B0BDE83040FCF7E4BC4449042222
:10D73000582003B0BDE83040FCF7DCBC414904226E
:10D74000742003B0BDE83040FCF7D4BC3E49012250
:10D75000652003B0BDE83040FCF7CCBC3B49042257
:10D76000402003B0BDE83040FCF7C4BC3849022279
:10D77000B22003B0BDE83040FCF7BCBC3549022202
:10D78000B02003B0BDE83040FCF7B4BC32490422FD
:10D79000702003B0BDE83040FCF7ACBC2F49042238
:10D7A000542003B0BDE83040FCF7A4BC2C49012252
:10D7B0006F2003B0BDE83040FCF79CBCC0B203B0A2
:10D7C000BDE83040FCF760BFF402FF1FF802FF1F06
:10D7D000C602FF1FFC02FF1FAC02FF1FA402FF1FB7
:10D7E000DC02FF1FE802FF1FBC02FF1FA002FF1F99
:10D7F0001003FF1F1203FF1FC002FF1FB802FF1F0D
:10D80000D402FF1F1403FF1F0A03FF1FE402FF1FC0
:10D81000C802FF1FC502FF1FCA02FF1FC402FF1F6D
:10D820000803FF1F0603FF1FEC02FF1FA802FF1FD4
:10D83000D802FF1F1803FF1FC902FF1F0503FF1FA8
:10D84000B402FF1FD002FF1FC102FF1F9C02FF1F77
:10D850000E03FF1F0C03FF1FCC02FF1FB002FF1FB0
:10D86000CB02FF1F38B5874CA378002B40F0C78050
:10D870006378403BBF2B00F21A81DFE813F0F5011B
:10D88000BF01B00118012C02DE010C029201180147
:10D890005402180183017401550164011801180133
:10D8A000260118014601180139011801CE0118019D
:10D8B00018011C021801180118011801180118019B
:10D8C0001801180118011801180118011801180190
:10D8D0001801180118011801180118011801180180
:10D8E0001801180118011801180118011801180170
:10D8F0001801180118011801180118011801ED018B
:10D900003C02A80149021C01180118011801180164
:10D91000180118011801180118011801180118013F
:10D92000180118011801180118011801180118012F
:10D93000180118011801180118011801180118011F
:10D94000180118011801180118011801180118010F
:10D9500018011801180118011801180118011801FF
:10D9600018011801180118011801180118011801EF
:10D9700018011801180118011801180118011801DF
:10D9800018011801180118011801180118011801CF
:10D9900018011801180118011801180118011801BF
:10D9A00018011801180118011801180118011801AF
:10D9B000180118011801180118011801180118019F
:10D9C000180118011801180118011801180118018F
:10D9D0001801180118011801180118011801110186
:10D9E000180118011801180118011801180118016F
:10D9F0001801180118011801180111010202012B68
:10DA000004D0022B17D0204B04221A700A280CD104
:10DA10001E4B1B784BB11C4B1D4A5B6813601D4AA3
:10DA200023B1136823F00803136038BD136843F073
:10DA30000803136038BD6378372B15D80A2800F027
:10DA40008281092819D00B2800F0FF810C28ECD125
:10DA50001149042240F21A7001EB830102FB03001A
:10DA6000BDE83840FCF720BB0C4A12889A421ED908
:10DA70000A2800F068810928D7D1074A616842F86E
:10DA8000231038BD2404FF1F1804FF1F0D04FF1FBF
:10DA9000D003FF1F7803FF1F3004FF1FFC11FF1F7F
:10DAA0000A28C2D1BE4ABF4B12785A60B0E7BD4BBC
:10DAB00003221A70AAE70A2800F04B810928B4D182
:10DAC000B84AB94B52681A6038BD0A2800F0508134
:10DAD0000928AAD1B54D21792B7DDA0702D5CB07CC
:10DAE00040F1CC8129751420BDE83840FCF7A6BA76
:10DAF0000A2800F04A81092897D16368012B40F277
:10DB0000C181A84B04221A7038BD0A2800F0428156
:10DB100009288AD1A549636841F8103F04221020E2
:10DB2000BDE83840FCF7E6BA0A2800F0178109285A
:10DB30007FF47BAF9D4A2379537519461520BDE8C4
:10DB40003840FCF77BBA0A2800F00D81092800F064
:10DB500078810B287FF469AF944B0720D979BDE811
:10DB60003840FCF76BBA0A2800F04D8109287FF491
:10DB70005CAF8E4A2379D37019460320BDE8384044
:10DB8000FCF75CBA0A2800F0228109287FF44DAF27
:10DB9000864A2379137119460420BDE83840FCF702
:10DBA0004DBA0A2800F0398109287FF43EAF7F4D35
:10DBB00063682946042241F8083F0820FCF79AFAD6
:10DBC0002A8A29896879BDE83840FBF717BA0A28FC
:10DBD0007FF42BAF764A734B12685A6018E70A2815
:10DBE00000F0F08009287FF420AF704A2379537049
:10DBF00019460120BDE83840FCF720BA0A2800F099
:10DC0000FD8009287FF411AF684A23791370194603
:10DC10000020BDE83840FCF711BA0A2800F0E48083
:10DC200009287FF402AF6149237901F8023F0122FC
:10DC30000220BDE83840FCF75DBA0A2800F0F78002
:10DC400009287FF4F2AE594A237953711946052009
:10DC5000BDE83840FCF7F2B90A287FF4E6AE554A31
:10DC6000504B12785A60D3E60A2800F0FA8009284F
:10DC70007FF4DBAE217940F2FF70BDE83840FCF75D
:10DC8000DDB90A2800F0A88009287FF4CEAE4A4BFF
:10DC900022791A7038BD0A2800F0BA8009287FF46A
:10DCA000C4AE4249636841F80C3F04220C20BDE831
:10DCB0003840FCF71FBA0A2800F09B8009287FF43F
:10DCC000B4AE3A49636841F8203F04222020BDE801
:10DCD0003840FCF70FBA0A2800F0A48009287FF426
:10DCE000A4AE3249636841F8183F04221820BDE809
:10DCF0003840FCF7FFB90A287FF497AE2D4B294A2C
:10DD00001B78A3F10403B3FA83F35B0953607FE646
:10DD10000A2800F0918009287FF487AE214A274B1A
:10DD200052681A6038BD0A2827D009287FF47DAED2
:10DD30002179002940F09C801C4B99751620BDE884
:10DD40003840FCF77BB91E49164A51F8233053601E
:10DD50005EE6154A134B12685A6059E6134A114B96
:10DD6000527D5A6054E6114A0E4BD2795A604FE602
:10DD70000E4A0C4B127D5A604AE60C4B094A9B7DB9
:10DD8000003318BF0123536042E6084A054BD27D99
:10DD90005A603DE6054A034B12695A6038E600BFF7
:10DDA0001C03FF1F1804FF1F0012FF1F2003FF1F8B
:10DDB0000404FF1F0E04FF1F0C04FF1F0412FF1FAB
:10DDC0003004FF1F344A354B52785A6020E6324AFD
:10DDD000324B12795A601BE6314B304A1B780033C4
:10DDE00018BF0123536013E62B4A2C4B92785A60DC
:10DDF0000EE6294A294B126A5A6009E6264A274B41
:10DE000012785A6004E6244A244BD2785A60FFE51F
:10DE1000214A224BD2685A60FAE51F4A1F4B92688A
:10DE20005A60F5E51C4A1D4B92695A60F0E51A4AA2
:10DE30001A4B52795A60EBE51A4A184B12685A602D
:10DE4000E6E5154B2279DA7138BD1749042240F214
:10DE50001A7001EB830102FB0300BDE83840FCF7B8
:10DE600049B940F2FF70FCF7CFF80C4B5860CFE592
:10DE7000094A0A4B0121917559605FE7FCF784FA62
:10DE800021792FE60449237901F8173F0122172051
:10DE9000BDE83840FCF72EB92003FF1F1804FF1F10
:10DEA0000C04FF1F0412FF1F3004FF1F074B9A785A
:10DEB000022A04D15A6858782AB9FAF7AFBF044B3E
:10DEC00004221A707047FAF7ABBF00BF2404FF1F8B
:10DED0001804FF1F38B5204B9A78012A20D017D399
:10DEE000022A0FD01D4B04221A701D4A127842B12B
:10DEF0001C4A5B6813601C4AC3B1136823F0080313
:10DF0000136038BD5878FAF78DFF144B5860ECE772
:10DF10005878FF280FD0FAF767FF104B5860E4E7F6
:10DF20005878FAF781FF0D4B5860DEE7136843F02D
:10DF30000803136038BD0120FAF756FF054600209C
:10DF4000FAF752FF44000220FAF74EFF44EA850434
:10DF5000024B20435860C8E72404FF1F1804FF1F2A
:10DF60000D04FF1FD003FF1F7803FF1F034B9A7898
:10DF700002B170475868404201F00EB92404FF1FF7
:10DF8000034B9A7802B17047586801F005B900BF99
:10DF90002404FF1F024B987800B1704701F0FCB8D1
:10DFA0002404FF1F0A4B9A7832B95A7862B1012AC9
:10DFB00006D1586801F04EB9064B04221A7070471A
:10DFC000044B03221A707047586801F013B900BF60
:10DFD0002404FF1F1804FF1F10B4124B5B789BB979
:10DFE0001149124B0868124A1249DB7802F8013BCA
:10DFF0000124431E0C70073013F8011F02F8011BA7
:10E000008342F9D110BC7047012BFBD10A4BC124CC
:10E01000602002210B22DC71987159711A7110BCB9
:10E02000704700BF2404FF1F1C00FF1F2003FF1FB9
:10E03000D803FF1FD403FF1F1804FF1FF8B50D49B5
:10E040000D4B01E08B4207D053F8042F0132F9D079
:10E050000A4B08221A70F8BD094C0A4F04F50066F5
:10E06000C4F5FE25281954F8041FB847B442F9D165
:10E07000F8BD00BFFCF70700FCEF07001804FF1F06
:10E08000F809FF1F9D2C01000C4A5378012B10D07A
:10E0900009D3FF2B06D15368094A03F5FE231B68F9
:10E0A0005360704770474FF4FE22054B12685A6068
:10E0B0007047044A024B12685A6070472404FF1FDD
:10E0C0001804FF1F04F007004FF0E02318B9044ABA
:10E0D000C3F80C2D7047034AC3F80C2D704700BFDE
:10E0E0000100FA050400FA05194A1A4938B51368FF
:10E0F00023F07F4323F0FF038B4203D0164B04220F
:10E100001A7038BD5268154B9A42F7D1FAF732FEB1
:10E1100072B6FBF7A3FC124C124B134D13484FF091
:10E12000E0214FF0FF32C3F88020C3F88021C3F80C
:10E130008420C3F88421C3F88820C3F88821C3F859
:10E140008C20C3F88C212560C1F80C0D38BD00BFB0
:10E150002404FF1F008192001804FF1FD6C5B4A33A
:10E160000000FF1F00E100E0785634120400FA05B9
:10E17000044B5A6840F2D2439A4202D1024B012228
:10E180001A7070472404FF1FF909FF1F10B52D4BAB
:10E1900098785A7882B040B1032A10D0042A4CD023
:10E1A000294B04221A7002B010BD0A2A41D8DFE8B8
:10E1B00002F012171C064421242E32373B0002AA1B
:10E1C000002142F8041D0146586802F0EFFA1E4B88
:10E1D000019A5A60E7E702F0E3FA1B4B5860E2E766
:10E1E00002F0DAFA184B5860DDE702F0DDFA164B60
:10E1F0005860D8E702F074FAD5E702F079FA0446DD
:10E2000002F07CFA104B2043C0B25860CBE758684C
:10E2100002F0E0FAC7E702F0FDFA0B4B5860C2E7E4
:10E22000586802F0FDFABEE702F000FB064B5860AA
:10E23000B9E7054B03221A70B5E7596802F042FAB4
:10E24000B1E700BF2404FF1F1804FF1F38B5054ABB
:10E25000054B1078546858706425411E1D705C6031
:10E2600004E000BF2404FF1F1804FF1FFE2900F272
:10E27000E081DFE811F0D501CC01C401C001BA0191
:10E28000BA01BA01BA01B601B601B601B601DE01A2
:10E29000B201AE01DE01DE01DE01AA01A601A2018A
:10E2A0009E019A019601DE01DE0192018E01DE01DE
:10E2B0008A01860182017E017A0176017201DE0106
:10E2C000DE016E01DE01DE01DE01DE01DE01DE01C6
:10E2D000DE01DE01DE01DE01DE01DE01DE01DE0146
:10E2E000DE01DE01DE01DE01DE01DE01DE01DE0136
:10E2F000DE01DE01680168016801680168016801EA
:10E3000068016801DE01DE01DE01DE01DE01DE0101
:10E31000DE01DE01DE01DE01DE01DE01DE01DE0105
:10E32000DE01DE01DE01DE01DE01DE01DE01DE01F5
:10E33000DE01DE01DE01DE01DE01DE01DE01DE01E5
:10E34000DE01DE01DE01DE01DE01DE01DE01DE01D5
:10E35000DE01DE01DE01DE01DE01DE01DE01DE01C5
:10E36000DE01DE01DE01DE01DE01DE01DE01DE01B5
:10E37000DE01DE01640160015C0158014C014301D2
:10E380003C01380134011D01DE01DE0119011501D6
:10E390001101DE01DE01DE01DE01DE01DE01DE0152
:10E3A000DE01DE01DE01DE01DE01DE01DE01DE0175
:10E3B000DE01DE01DE01DE01DE01DE01DE01DE0165
:10E3C000DE01DE01DE01DE01DE01DE01DE01DE0155
:10E3D000DE01DE01DE01DE01DE01DE01DE01DE0145
:10E3E000DE01DE01DE01DE01DE01DE01DE01DE0135
:10E3F000DE01DE01DE01DE01DE01DE01DE01DE0125
:10E40000DE01DE01DE01DE01DE01DE01DE01DE0114
:10E41000DE01DE01DE010D010901DE01DE01DE01AA
:10E42000DE01DE01DE01DE01DE01DE01DE01DE01F4
:10E43000DE01DE01DE01DE01DE01DE01DE01DE01E4
:10E44000DE01DE01DE01DE01DE01DE01DE01DE01D4
:10E45000DE01DE01DE01DE010501DE01DE01DE019D
:10E46000DE01DE01DE01DE01DE01DE01DE01DE01B4
:10E47000DE01FF0040F2D2439C4200F0DD8038BD57
:10E48000BDE83840FFF730BEBDE83840FFF7FCBDBF
:10E49000BDE83840FFF7D2BDBDE83840FFF776BE93
:10E4A000BDE83840FCF746BFBDE83840FDF7FAB993
:10E4B000116821F07F4121F0FF010029DFD140F2F6
:10E4C000D2439C42DBD140F2FF70FBF7B7FDFBF774
:10E4D0005BFF4FF0E0235A4AC3F80C2D38BDBDE86E
:10E4E0003840FFF779BDBDE83840FDF7CBB8554B54
:10E4F000197DD878BDE83840FDF778B9FDF7BCF84C
:10E50000FAF720FC0020BDE8384000F0C9BEFAF759
:10E5100031FC4C4B1C7DFBF715FD01462046BDE848
:10E520003840FDF78DB8BDE83840FCF7DDBEBDE8EA
:10E530003840FCF7D3BEBDE83840FCF7BDBEBDE8AF
:10E540003840FCF7F1BE404A4049BDE83840FAF790
:10E5500047BDBDE83840FCF787BEBDE83840FDF751
:10E5600015B8BDE83840FCF79BBEBDE83840FCF765
:10E570006DBEBDE83840FCF795BFBDE83840FDF7FB
:10E58000A3BABDE83840FDF769BABDE83840FDF7E9
:10E590004BBABDE83840FDF7B1B9BDE83840FDF7EA
:10E5A000DFB9BDE83840FDF76BB9BDE83840FDF78D
:10E5B00003B9BDE83840FDF79DB8BDE83840FDF728
:10E5C000A3B8BDE83840FDF713B8BDE83840FCF704
:10E5D0000BBFBDE83840FFF77DBCBDE83840FFF712
:10E5E00065BCBDE83840FFF73DB9174A1749BDE89B
:10E5F0003840FDF75BBDBDE83840FFF7D3BC9078ED
:10E6000000287FF43CAFBDE8384000F0C5BD9378EA
:10E61000002B7FF434AF6042BDE8384000F0BCBD51
:10E620009378002B7FF42BAF2046BDE8384000F0F4
:10E63000B3BD02221A7022E7054B01221A7038BDC1
:10E640000400FA052003FF1F1804FF1F2404FF1F06
:10E65000F909FF1F2DE9F047BD4B1B7886B0054631
:10E66000F3B9BC4B1B78DBB9BB4CBC4E23785A1EAC
:10E67000012A40F2388102AF032B40F0DA80337870
:10E68000002B00F09181012B14D1DFF8048308F1F5
:10E69000090918F8010FFAF787FFC145F9D109E018
:10E6A000AF4B1B78063BDBB2192B40F28780AA4C9C
:10E6B000AA4E02AFAB4BDFF89C821A78002388F891
:10E6C00000302370337022B14FF0E023A64AC3F824
:10E6D0000C2D3846FAF71EFD0746002875D0A04BD2
:10E6E000A24A9DF810601E7012699DF811009DF8F5
:10E6F0001260039958709E709DF813009DF8146085
:10E70000D87191429E719DF815009DF81660587160
:10E710001E7104BF012388F800309DF80830944E24
:10E720009DF809006070072B0CBF012302232370A2
:10E7300033785A1E012A40F22D81052B00F02A81E0
:10E740008C4B01221A700DF10700FAF747FF0028E1
:10E7500000F0B8800127FAF75BFF002840F0AB809B
:10E76000A2789DF80710531CDBB22244092BA3703A
:10E77000117140F0A5807D4B21795A78A0708A42B2
:10E780009B7800F07581002B00F09C80994240F04E
:10E790009980012388F80030774A0023D01D01E0DA
:10E7A00012F8011B0B449042DBB2F9D1227B9A4252
:10E7B00000F0708104232370337812E06F4A22FA4C
:10E7C00003F3D9073FF550AF71E70DF10700FAF7F2
:10E7D00005FF674E0028BED133785A1E012A40F249
:10E7E0002E81042B71D02278082A5CD9FFF72EFDE8
:10E7F0002378092B1AD13378022B00F01481604B57
:10E80000186898B13378012B10D15E4B5E4A1C68B2
:10E8100013689C4218BF002305D126E152F8041F5B
:10E820008C4200F0228101339842F7D806B0BDE84F
:10E83000F087042B7FF43EAFDFF830A1DFF84C8186
:10E840009AF803009AF801900023012288F800202A
:10E8500088F80130C8F804308144FAF7A5FE9AF828
:10E860000100FAF7A1FE98F80000FAF79DFE98F86B
:10E870000100FAF799FE98F80700FAF795FE98F864
:10E880000600FAF791FE09F1010998F80500FAF778
:10E890008BFE5FFA89F998F80400FAF785FE48467E
:10E8A000FAF782FE06E740F25113D340DA079DD50E
:10E8B00006B0BDE8F08701229DF80730A2702371F1
:10E8C000002F89D03378042B8DD1254B93F900305C
:10E8D000002B88DB01F0B8FA2278082A40F2A680E3
:10E8E000FDF712F8A2E721493278C8680390012B9E
:10E8F0000CBF0723082360788DF8083000238DF8BB
:10E9000009008DF80A30002A48D1204B896893F815
:10E9100000E05F78D8798DF810108DF8172099797C
:10E920005A791B798DF811E08DF812708DF813006B
:10E930008DF814108DF815208DF8163002AF38467A
:10E94000FAF75CFC00283FF471AF237894E600BF2F
:10E950000C04FF1FF809FF1FE001FF1FD403FF1F76
:10E960002404FF1FF909FF1F0400FA052003FF1FFD
:10E970000E04FF1F0D04FF1FE501FF1F110200021F
:10E98000F409FF1F0404FF1FCC09FF1F1804FF1F19
:10E99000D703FF1F524B00221A70D4E6012A59D028
:10E9A000022ACBD102AF85E6DFF84CA1DFF84C910B
:10E9B0009AF803009AF8018099F8002099F801303C
:10E9C0008044904499F80720984499F80630904480
:10E9D00099F80520984499F8043090449844FAF73F
:10E9E000E3FD9AF80100FAF7DFFD99F80000FAF765
:10E9F000DBFD99F80100FAF7D7FD99F80700FAF75F
:10EA0000D3FD99F80600FAF7CFFD99F80500FAF75B
:10EA1000CBFD5FFA88F899F80400FAF7C5FD404687
:10EA2000FAF7C2FD46E605233370E8E640F25113DB
:10EA3000D340DB077FF554AF06B0BDE8F087012D6A
:10EA40007FF4D1AE274B1868B0F5006F14D90023BE
:10EA50003370C8E6244B04AA03F1080013F8011B25
:10EA600002F8011B8342F9D168E705233370DDE624
:10EA70008B427FF491AE8CE6421C1C491A60FBF776
:10EA8000E5FB174A3378157009222270042B7FF4B6
:10EA9000ADAE1AE7154B6179A279257A19705A70D3
:10EAA000A17AE27AE779607ADD7159711A719F7003
:10EAB0009871FAF7D9FF0E4A337810600D4D5A1E3F
:10EAC00000200321012A28702170054A04D9052B52
:10EAD00002D001211170D9E700211170D6E700BFE3
:10EAE0000D04FF1F0404FF1FD903FF1F2404FF1F91
:10EAF0001404FF1F2004FF1F2003FF1F1804FF1F23
:10EB0000F0B50246264B007992F801C092F802E077
:10EB1000D678D87150799871224C9E700D469179B3
:10EB2000597194E80300D7791F4A83F800C083B075
:10EB300083F801E01F71002313708DE80300FFF7D5
:10EB400085FB1A4B1B786E46B3B1012B05D096E8B6
:10EB5000030084E8030003B0F0BD154A6B1E0735BF
:10EB600012F8011B03F8011FAB42F9D196E803002C
:10EB700084E8030003B0F0BD2B706B7063782278DB
:10EB8000AA70EB70E3792B71A3796B716379AB7128
:10EB900096E803002379EB7184E8030003B0F0BD2D
:10EBA0002404FF1F1804FF1F0D04FF1FD403FF1FC1
:10EBB000D903FF1F08B50C4B196821F07F4121F0E4
:10EBC000FF0121B95A6840F2D2439A4200D008BDF1
:10EBD00040F2FF70FBF732FAFBF7D6FB4FF0E02371
:10EBE000024AC3F80C2D08BD2404FF1F0400FA05D7
:10EBF00010B50D4CFAF7FEFD94F82920E36B214681
:10EC00005208B3FBF2F3B0FBF3F202FB130021F85E
:10EC1000400F02228020FBF76DFA94F8423023F077
:10EC2000010384F8423010BD9C02FF1F10B5064C52
:10EC3000B4F84000FAF7F0FD94F8423023F00203F4
:10EC400084F8423010BD00BF9C02FF1F38B5002081
:10EC5000FAF758F90B4B93F82520092A054602D9F3
:10EC6000094C257038BD40F24123D340DB07064CE8
:10EC7000F7D501462078FAF78FFE636825701844AF
:10EC8000606038BD9C02FF1FF001FF1F094B684602
:10EC9000D3F8A02020F007018D46520601B406D516
:10ECA0009A69054942F0807201209A61087201BC9C
:10ECB0008546704700A00440F001FF1F1A4B6846CC
:10ECC000D3F8A02020F007018D46910601B503D4AA
:10ECD000D3F8A020120617D5FFF7B8FF0020FAF7E7
:10ECE00011F904281BD0104B5A6942F080725A6106
:10ECF000DA6942F08072DA611A6A42F080721A624E
:10ED0000BDE8014085467047D3F8A030DB05F7D554
:10ED1000FFF79CFF0020FAF7F5F80428E3D1012162
:10ED20000220FAF70DF8DEE700B004400346044A7B
:10ED300000EBD070C0F34F0082F82930FAF73ABDEB
:10ED40009C02FF1F01280CD007D3022803D1074BD8
:10ED5000B3F90400704700207047044BB3F900007A
:10ED60007047024BB3F90200704700BF6812FF1FE3
:10ED7000F9F7E8BF00B585B001F0BAFC10B905B0ED
:10ED80005DF804FB01F046FD0328F8D10020FAF7F6
:10ED90004BF800900120FAF747F801900420FAF7A9
:10EDA00043F802900520FAF73FF804AB039013E90B
:10EDB0000F0001F0BFFCE2E770B50A4C0A4DE069B4
:10EDC00002F0C0FD0146094802F0C8FE064694F86C
:10EDD000290002F0B7FD0146304602F0BFFE286070
:10EDE00070BD00BF9C02FF1F2C00FF1F0050C348D6
:10EDF00070B5094C094DE06902F0A4FD01460848D0
:10EE000002F0ACFE0646E06B02F09CFD0146304687
:10EE100002F0A4FE686070BD9C02FF1F2C00FF1F63
:10EE2000007C924938B5054600200C46FAF76AF88E
:10EE3000314B93F8283013B180F00700C0B214B9F9
:10EE400080F00700C0B22D4B0022C3F890200728A5
:10EE50000FD8DFE800F01D212B313C47041D274B64
:10EE600027490C24002202201C66C8609D619A621A
:10EE70009A63224B9A6D4FF4007042F004029A6537
:10EE80000021C3F898000220BDE83840F9F758BFC8
:10EE90001A4B3F221A66ECE7184B194900220C2046
:10EEA0001866CA609A619A629D63E2E7134B14493F
:10EEB000302400220120D7E7104B114900220324FF
:10EEC00001201C66C8609A619A629D63D1E70B4B72
:10EED0000B490022032402201C66C8609A619D62CF
:10EEE0009A63C6E7054B0649002230201866CA60BF
:10EEF0009A619D629A63BCE79C02FF1F00800340F9
:10EF0000F001FF1FF8B55748574C584E01F016FF57
:10EF1000574801F013FF574801F010FF94F82500FF
:10EF2000FAF7DAFDE06902F00DFD014605465248A8
:10EF300002F014FE074694F8290002F003FD014692
:10EF4000384602F00BFE294630604C4802F006FEBF
:10EF50000546E06B02F0F6FC0146284602F0FEFD95
:10EF600094F825507060062D30D0072D3CD0082D28
:10EF70005ED0092D12D06DB94FF40040FAF7B4FFFE
:10EF80008020FAF7B9FF0120FAF7A6FC29462846A7
:10EF9000FFF748FFBDE8F840F9F7D4BE4FF4004052
:10EFA000FAF7A2FF8020FAF7A7FF0120FAF794FCF6
:10EFB00094F82D10E06BFAF79FFB94F82910E06BA2
:10EFC0004908FAF7EDFB94F82550D4E74FF40040D8
:10EFD000FAF78AFF8020FAF78FFF0120FAF77CFC0E
:10EFE00094F82550072DC2D14FF40040FAF784FF62
:10EFF0008020FAF781FF94F82C30012B2DD094F863
:10F000002D10E06BFAF778FB94F82910E06B4908B3
:10F01000FAF7C6FBFAF70EFCFCF758F80120FAF7EE
:10F020000FFC94F82550164B0022082D1A72A0D11F
:10F030004FF40040FAF758FF0020FAF74DFC94F81F
:10F040002D10E06BFAF758FB94F82910E06B490893
:10F05000FAF7A6FB94F825508BE70020FAF73CFC62
:10F06000CDE700BF3012FF1F9C02FF1F2C00FF1FC7
:10F070009812FF1F1012FF1F0050C348007C9249D6
:10F08000F001FF1F014B01221A747047F001FF1FAE
:10F09000B0F5007F10B504464AD02CDDB0F5806F86
:10F0A0001CD0B0F5006F16D1FAF71EFF4FF4807038
:10F0B000FAF722FF4FF48060FAF71EFF4FF400705A
:10F0C000FAF71AFF4FF48040FAF716FF1D4BA3F82A
:10F0D0006640F9F72BFE1C4B1C6010BDFAF704FFCD
:10F0E0004FF48070FAF708FF4FF40070FAF704FF4E
:10F0F0004FF40060E4E7B0F5807FECD1FAF7F4FE5E
:10F100004FF48060FAF7F8FE4FF40070FAF7F4FE5F
:10F110004FF40060FAF7F0FE4FF48040FAF7ECFE8F
:10F12000084BA3F86640F9F703FE074B1C6010BDBF
:10F13000FAF7DAFE4FF48070FAF7DEFE4FF48060E3
:10F14000D4E700BF9C02FF1F5812FF1F08B50F4BEA
:10F1500093F8252012B993F8692082B90C4A9B6F65
:10F16000000290FBF3F010604FF40060FFF790FF97
:10F17000084B00221A60F9F7E5FD012008BD044A9A
:10F18000DB6F000290FBF3F01060EDE79C02FF1FC5
:10F190006012FF1F9012FF1F00F54333104A03F562
:10F1A000A073934201D9002070470E4A0E4B10B550
:10F1B000146818604FF40070FFF76AFFB4F5006F31
:10F1C00003D0F9F7BFFD012010BD084B084C1868AB
:10F1D00002F0BCFB2060F9F7B5FD012010BD00BFB7
:10F1E000801A06005812FF1FC812FF1F5412FF1F7B
:10F1F0009012FF1F124A134B10B550611C684FF458
:10F200008060FFF745FF4FF48040FAF775FEB4F5D4
:10F21000007F0CD0B4F5006F05D10B4B0B4C186878
:10F2200002F094FB2060BDE81040F9F78BBD084A5E
:10F23000064B12681A60BDE81040F9F783BD00BFA5
:10F24000F001FF1F5812FF1F5412FF1F0812FF1F6B
:10F250009012FF1F024B5B681844FFF7CBBF00BF43
:10F26000F001FF1F0C4B93F8252012B993F8692089
:10F2700042B90A4A9B6F106800FB03F0002808DBC4
:10F2800000127047054ADB6F106800FB03F000288E
:10F29000F6DAFF30001270479C02FF1F5012FF1F6A
:10F2A00000F5AF33034A03F5C873934200D84DE726
:10F2B0000020704720BF0200014B5869704700BF13
:10F2C000F001FF1F08B5024B186802F059FD08BD98
:10F2D0009012FF1F014B9869704700BFF001FF1F9C
:10F2E000014BD869704700BFF001FF1F10B5164BE6
:10F2F000164C1878F9F798FD4FF4C673144A03FBBF
:10F3000000F082FB00320244C017C0EBE230B0F5DF
:10F310008C7FA0614FF004000ADBFAF7E5FDA369DA
:10F320003C2B4FF002000ADDBDE81040FAF7E4BDC7
:10F33000FAF7E2FDA3693C2B4FF00200F4DCBDE8D4
:10F340001040FAF7D1BD00BF1700FF1FF001FF1FEB
:10F350000180008010B5444B444C1878F9F764FDE7
:10F36000C0F30F1002F0F2FA01F0E2FE02460B4683
:10F3700031A1D1E9000102F059F831A3D3E900230A
:10F3800001F076FD02F0D8F9394902F0E7FB01F00F
:10F39000CFFE02F08FFF2CA3D3E9002301F01CFF66
:10F3A0002BA3D3E9002301F065FD02460B462AA1F9
:10F3B000D1E9000102F03AF829A3D3E9002301F0D2
:10F3C00057FD02F0B9F902F0DBFCE0610820FAF722
:10F3D000A7FDE36948B9772B4FF0080022DCFAF764
:10F3E0008BFDF9F7F7FC48B110BD6D2BFCDC082054
:10F3F000FAF782FDF9F7EEFC0028F5D1FAF7ACFD3B
:10F400000028F1D14FF40050FAF78AFD0028EBD123
:10F410004FF48070FAF784FD0028E5D1BDE8104074
:10F42000F9F790BCFAF760FDF9F7A4FC4FF480708F
:10F43000BDE81040FFF72CBE9A9999999999C1405F
:10F440009A999999999901400000000000A0724092
:10F450000000000000D4AA4000000000C83A2F417C
:10F4600000000000001071401600FF1FF001FF1F98
:10F470000000204138B5484CFAF7F6FA236AC31A5F
:10F48000002BB8BF5B42B3F57A7F56DAFFF72EFF49
:10F49000FCF7EAFB237A414D1BB195F82530072B89
:10F4A00052D0FBF7A3FEAB6D98422DD8FAF7DCFAE9
:10F4B000A36AEA6DC01A0028B8BF404290420ED33A
:10F4C00095F86420012A03D001F018F998B938BDE5
:10F4D0000023334985F86430A420FAF70BFE95F831
:10F4E0006430012BF0D14FF40030FAF7FDFC01F04D
:10F4F00005F90028EBD02B4A2B4B1068196862687D
:10F50000BDE8384001F098B9FAF7AEFA636AC01A5C
:10F510000028B8BF4042B0F57A7FC7DBFBF7F6FDA5
:10F520004FF40030FAF7E0FC95F864303BB3FBF79A
:10F530006FFEFAF799FA6062B8E70546FCF7A6FB9A
:10F54000FFF708FF2562A1E795F84230DA0703D5F7
:10F55000FFF74EFB95F84230980701D5FFF766FBA1
:10F5600095F85430D90707D5002262605A0703D5B1
:10F5700023F0010385F854300023237291E701231F
:10F580001A46074985F86430A420FAF7B3FDFAF764
:10F590006BFAA062CBE700BFF001FF1F9C02FF1FC8
:10F5A0000003FF1F5C12FF1F5412FF1F014B58681E
:10F5B000704700BFF001FF1F014B1868704700BF84
:10F5C000C812FF1F2DE9F041414C94F8253082B05C
:10F5D0000546092B25D8DFE803F03224242424240F
:10F5E00032052732FAF706F9E16B3A4C8A1090425D
:10F5F00002EB4206A36B2CDA9E422ADAC31A0B44B2
:10F60000354E61683268A063C91AD01A30606160F3
:10F6100013B1324A5B429360002D3FD0304BE26A17
:10F620001A6002B0BDE8F0812E4B186802F0A8FB0A
:10F630002B4A284B1060D86202B0BDE8F08178B147
:10F64000244B274A5868D96A1863116002B0BDE894
:10F65000F081B04220DD9A421EDDC31A5B1ACFE76B
:10F660001C4C1F4D236B60682E68C01A02F06EF9A7
:10F670001A4B196802F0BEF902F082FB082301461A
:10F6800000933246052304F1340001F0EDF963687C
:10F690002860E0622363C4E7C31AB1E702F056F9B9
:10F6A0000E4B0F4F5968D7F8008002F0A3F902F013
:10F6B00067FB08230146424600930B48022301F0F2
:10F6C000D3F90A4B32683860E0621A603560A8E707
:10F6D0009C02FF1FF001FF1FB812FF1F2C00FF1F2D
:10F6E0005412FF1F9012FF1F2402FF1F6412FF1FFE
:10F6F00008B50120FFF766FFFFF704FC0120FFF7C4
:10F7000061FF034A034B92F825201A7308BD00BF1E
:10F710009C02FF1F2C00FF1F044A054B92F8252076
:10F720001B7B9A4200D0E3E7704700BF9C02FF1F9B
:10F730002C00FF1FF8B50B4B0B4F58680B4E0C4DB0
:10F740000C4C0D4958610022002301203B603360BE
:10F750002B6022600A60FFF735FFBDE8F840FFF735
:10F76000D1BB00BFF001FF1FC812FF1F5012FF1FC7
:10F770006012FF1F0812FF1F9012FF1F10B50446F2
:10F780004FF48040FAF7B8FB034B01205C605C61EA
:10F79000BDE81040FFF716BFF001FF1F014B1868CE
:10F7A000704700BF5412FF1F0C4B93F8252012B96D
:10F7B00093F8692042B90A4A986F136800FB03F076
:10F7C000002808DB00127047054AD86F136800FB59
:10F7D00003F00028F6DAFF30001270479C02FF1F8A
:10F7E0005C12FF1F034A92F8423023EA000082F8BD
:10F7F000420070479C02FF1F034B93F842301842AF
:10F8000014BF0120002070479C02FF1F034A92F89A
:10F81000543023EA000082F8540070479C02FF1F16
:10F82000034B93F85430184214BF01200020704756
:10F830009C02FF1F014B1868704700BF7012FF1F2A
:10F84000684620F007018D462DE9F147B94D8FB08C
:10F8500001210020F9F774FA95F82530002B35D1F5
:10F86000B54CB64AB4F93C1081EAE173A3EBE173FD
:10F870009B10D360136843F001031360B048226CFF
:10F880000168636C21F080010160217C0132013349
:10F890002264636451B1AB4A95F82510127B914202
:10F8A00002D0FFF725FF636C00222274EA699A42B6
:10F8B00040D92A6A236C9A4211D900210846F9F7E7
:10F8C0003FFA0FB0BDE8F147854670479B4B9A4C15
:10F8D0000022DA601A6842F001021A60CEE70023C3
:10F8E000236401F095FA4FF48060FAF719FB0028C1
:10F8F00000F03E8195F82560002E40F0668195F875
:10F900006930012B00F0838008A8FAF731FBE26828
:10F910008D4B0898BDF824109980012A186000F0DA
:10F92000FB81022A00F0F481002A73D11E887642FE
:10F9300036B26FE00026854F666401F07FFA3046EC
:10F94000FFF740FE3A682B6982EAE271A1EBE271AF
:10F9500083EAE372A2EBE37291424FF0100053DDB1
:10F96000FAF7CAFA4FF48060FAF7DAFA002840F0A2
:10F97000858195F82430012B00F0A4812A68744B0E
:10F98000744E1868514201F02DF801F0DFFF30602D
:10F990004FF40070FAF7C4FA002800F0678195F878
:10F9A0002530002B40F0B98095F86930002B00F02D
:10F9B000B4806B68EE6F1B0293FBF6F6DFF8948160
:10F9C000D7F80090D8F8000002F0DAF9334649463B
:10F9D000614AFAF781FE614B186000F089FE002849
:10F9E0003FF467AF00F016FF01287FF462AFD8F84C
:10F9F000000002F0C5F93B680B930A900EAB13E9C7
:10FA00000F0000F097FE54E7FAF76EFAAAE7FAF74C
:10FA1000E7FA06B294F84830012B95F8693004BF34
:10FA2000764236B2002B7ED06B68EA6F1B0293FBE6
:10FA3000F2F34A4F4A4A38683146FAF7C7FE494B53
:10FA40003A68A08700281A60C0F25781002384F822
:10FA50004830454F45483A6808233146009304230F
:10FA600001F002F8B4F93C30386083EAE37094F8AE
:10FA70004810A0EBE370FFF7D5F900F039FE00283D
:10FA800040F09280FFF776F995F82530002B40D1B1
:10FA900095F86930002B3CD039686B68EA6F81EAD1
:10FAA000E176A6EBE1761B0293FBF2F39E42D4BF14
:10FAB0000026012631460120FAF726FA3046F9F7EA
:10FAC00033F995F86A3053B1A269B5F86C309342B6
:10FAD00040F31781B5F86E105B1A9A4205DAF9F710
:10FAE00087FA4FF48020FAF707FAFFF75DFEFBF77D
:10FAF00015FB4FF40030FAF713FA002850D1F9F74C
:10FB000069F900287FF4D9AE4FF48070FFF7C0FA8E
:10FB1000D3E639686B68AA6FC1E76B68AE6F1B02EA
:10FB200093FBF6F64AE76B68AA6F1B0293FBF2F3AE
:10FB30007FE700BF9C02FF1FF001FF1F0060034032
:10FB4000008003402C00FF1F6812FF1F5412FF1F8C
:10FB5000C812FF1F9012FF1F3012FF1F6012FF1FFD
:10FB60009812FF1F5012FF1F5C12FF1F3C02FF1F65
:10FB70004FF40070FAF7D4F900287FF4BBAE4FF4CD
:10FB80000060FAF7CDF9064600287FF4B3AE4FF4D3
:10FB90008070FAF7C5F9002840F0DC807C4F73E7ED
:10FBA0000020FFF7D3FAAAE700F034FE00287FF424
:10FBB00069AFFFF757FB0A90FFF7F6FD0EAB0B900E
:10FBC00013E90F0000F0B6FD5CE7DFF8FCA1714E11
:10FBD000DFF8F891DFF8F8816D4F08A8FAF7C8F957
:10FBE000089A6D48BDF82430CAF800206B496A684D
:10FBF0000068AAF804300968BAF804E00690120216
:10FC0000A86F92FBF0F266480792664ADAF8003075
:10FC1000ADF800E0059104900392CDF80490624A9B
:10FC2000624963480296FAF777FE624BD9F800E022
:10FC3000C3F800E04FF00809B6F90010D8F800202A
:10FC40005D48CDF80090022300F00EFFB6F90230B7
:10FC5000B6F90010C8F800003A685848CDF800908E
:10FC60001944042300F000FF386006E74FF4806079
:10FC7000FAF756F900287FF492AE1AE6504A616806
:10FC80006069FAF707FD454B186000F031FD002868
:10FC900046D163696168EA68591A81EAE173A3EBA6
:10FCA000E17393423FF765AE3B68AA6883EAE3716C
:10FCB000A1EBE37191423FF75CAE4FF48040FAF75D
:10FCC00013F956E64FF48060FAF72AF9002835D187
:10FCD0004FF40070FAF724F900283FF459AE2F4B87
:10FCE0002F4ED3F80080306802F04AF84146FAF708
:10FCF000BDFB01F02BFE30604AE6012384F848305A
:10FD0000A7E6F9F76FF94FF48020FAF7EDF8ECE683
:10FD10009E88764236B27DE65E88764236B279E6D5
:10FD200000F078FD0228B4D1626963680B930A92EF
:10FD30000EAB13E90F0000F0FDFCAAE7174A636958
:10FD4000116818486268164EFAF7D2FB01F0FEFD02
:10FD50003060BDE714480E4F00F0F0FF184800F087
:10FD6000EDFF134800F0EAFF104800F0E7FF0C4BEE
:10FD7000104995F825000E6000221A603E60F9F7E0
:10FD80007DFF104B4FF40072C3F898207AE600BF55
:10FD90005C12FF1FBC12FF1F5412FF1FC812FF1F6F
:10FDA0009012FF1F0812FF1F3012FF1F1012FF1FBB
:10FDB0009812FF1F5012FF1F4002FF1F4402FF1F37
:10FDC0007012FF1F008003406812FF1F6012FF1FA8
:10FDD000C012FF1F684620F007018D4601B5F8F7F5
:10FDE00095FF044ABDE80140136823F04003136007
:10FDF0008546704700600340034B93F84230DB07B1
:10FE000001D5FEF7F5BE70479C02FF1F034B93F828
:10FE100042309B0701D5FEF709BF70479C02FF1FC8
:10FE2000074A92F85430D80708D5064900204860A0
:10FE3000590744BF23F0010382F85430704700BFD4
:10FE40009C02FF1FF001FF1F08B5F8F793FF4FF466
:10FE50008070BDE80840FFF71BB900BF014B186870
:10FE6000704700BF3012FF1F014B9868704700BFFA
:10FE70003012FF1F014B1868704700BF9812FF1F18
:10FE8000014B9868704700BF9812FF1F014B18681C
:10FE9000704700BF1012FF1F014B9868704700BFEA
:10FEA0001012FF1F014B5868704700BF9C02FF1FD4
:10FEB000044A904298BF044A03469ABF5360012007
:10FEC00000207047905F01009C02FF1F014B986B60
:10FED000704700BF9C02FF1F044A904298BF044A2B
:10FEE00003469ABF9363012000207047905F010092
:10FEF0009C02FF1F014B93F8290070479C02FF1FD3
:10FF0000831EFC2B02D900231846704770B50E4C97
:10FF10000E4D84F82900C0F34F00F9F74BFCE0695F
:10FF200001F010FD01460A4801F018FE064694F85B
:10FF3000290001F007FD0146304601F00FFE0123C4
:10FF40002860184670BD00BF9C02FF1F2C00FF1FD9
:10FF50000050C3480030034B18BF012083F828002D
:10FF6000704700BF9C02FF1F034B93F8280000302E
:10FF700018BF0120704700BF9C02FF1F012898BFD7
:10FF8000034A03469ABF82F82E30012000207047B2
:10FF90009C02FF1F014B93F82E0070479C02FF1F2D
:10FFA000B0F5803F0BD208B5064BDA6BD8639042B0
:10FFB00003D0FFF7BFFB012008BD012008BD0020D2
:10FFC000704700BF9C02FF1F014BD86B704700BFFA
:10FFD0009C02FF1FB0F5803F38BF044A03463ABF7A
:10FFE000A2F8403001200020704700BF9C02FF1F94
:10FFF000014BB3F8400070479C02FF1F064B0030D6
:020000021000EC
:1000000093F82D2018BF0120824283F82D0001D0E3
:10001000FFF790BB704700BF9C02FF1F034B93F894
:100020002D00003018BF0120704700BF9C02FF1F49
:10003000022898BF034A03469ABF82F82C30012059
:10004000002070479C02FF1F014B93F82C00704763
:100050009C02FF1F00F54333054903F5A0738B4253
:1000600098BF044B02469ABF1A66012000207047D1
:10007000801A06009C02FF1F014B186E704700BFDC
:100080009C02FF1F42F21072904298BF034A03463F
:100090009ABF538501200020704700BF9C02FF1FBC
:1000A000014BB3F92A0070479C02FF1F831F032BEB
:1000B00000D930B9044A054B82F825000120187494
:1000C00070470020704700BF9C02FF1FF001FF1F18
:1000D000014B93F8250070479C02FF1F094BB3F8B2
:1000E0006630B3F5806F08D0B3F5006F07D0B3F575
:1000F000007F0CBF022000207047032070470120C2
:10010000704700BF9C02FF1F0A2898BF034A03469E
:100110009ABF136201200020704700BF9C02FF1F9E
:10012000014B186A704700BF9C02FF1FB0F5803F6B
:1001300038BF034A03463ABF1363012000207047CB
:100140009C02FF1F014B186B704700BF9C02FF1FF2
:10015000B0F5803F38BF034A03463ABF53630120DE
:10016000002070479C02FF1F014B586B704700BF77
:100170009C02FF1F044A904298BF044A03469ABF5C
:100180005361012000207047400D03009C02FF1FB7
:10019000014B5869704700BF9C02FF1F044A904200
:1001A00098BF044A03469ABF13600120002070479D
:1001B000400D03009C02FF1F014B1868704700BFF1
:1001C0009C02FF1F044A904298BF044A03469ABF0C
:1001D0001361012000207047400D03009C02FF1FA7
:1001E000014B1869704700BF9C02FF1F1428F8B527
:1001F00023D8134C134DE06101F0A4FB01460646E1
:10020000114801F0ABFC074694F8290001F09AFB75
:100210000146384601F0A2FC314628600B4801F047
:100220009DFC0646E06B01F08DFB0146304601F077
:1002300095FC012368601846F8BD00231846F8BDF8
:100240009C02FF1F2C00FF1F0050C348007C9249F6
:10025000014BD869704700BF9C02FF1FB0F5803F7B
:1002600038BF034A03463ABFD364012000207047D9
:100270009C02FF1F014BD86C704700BF9C02FF1F00
:10028000B0F5803F38BF034A03463ABF13650120EB
:10029000002070479C02FF1F014B186D704700BF84
:1002A0009C02FF1F012898BF034A03469ABF82F8A9
:1002B00024300120002070479C02FF1F034B93F85D
:1002C0002400003018BF0120704700BF9C02FF1FB0
:1002D000044A904298BF044A03469ABF93610120A2
:1002E00000207047A08601009C02FF1F014B986907
:1002F000704700BF9C02FF1FB0F5803F38BF034A24
:1003000003463ABF93640120002070479C02FF1F00
:10031000014B986C704700BF9C02FF1F044A90423B
:1003200098BF044A03469ABF93600120002070479B
:10033000400D03009C02FF1F014B9868704700BFEF
:100340009C02FF1F044A904298BF044A03469ABF8A
:10035000D360012000207047A08601009C02FF1F8F
:10036000014BD868704700BF9C02FF1F064A92F8F5
:10037000543020B923F0010382F85430704743F021
:10038000010382F8543070479C02FF1F024B93F820
:10039000540000F0010070479C02FF1F064A92F8CB
:1003A000543020B923F0040382F85430704743F0EE
:1003B000040382F8543070479C02FF1F024B93F8ED
:1003C0005400C0F3800070479C02FF1F012898BFB3
:1003D000034A03469ABF82F86A3001200020704722
:1003E0009C02FF1F014B93F86A0070479C02FF1F9D
:1003F000A0F13202B2F5D77F98BF044A03469ABFF4
:10040000A2F86C3001200020704700BF9C02FF1F43
:10041000014BB3F86C0070479C02FF1F322898BF55
:10042000034A03469ABFA2F86E30012000207047AD
:100430009C02FF1F014BB3F86E0070479C02FF1F28
:10044000044A904298BF044A03469ABFD3650120EC
:1004500000207047E09304009C02FF1F014BD86D01
:10046000704700BF9C02FF1F044A904298BF044A95
:1004700003469ABF936501200020704780DF171064
:100480009C02FF1F014B986D704700BF9C02FF1F2D
:10049000012898BF034A03469ABF82F869300120B9
:1004A000002070479C02FF1F034B93F86900003047
:1004B00018BF0120704700BF9C02FF1F08B54FF610
:1004C000FE73984201D9002008BD03460549064A3B
:1004D00008789BB21946A2F87030F8F7EFFC0120BB
:1004E00008BD00BF1000FF1F9C02FF1F014BB3F8A7
:1004F000700070479C02FF1FB0F5805F01D30020A1
:10050000704708B5034BA3F87200F8F7A9FA012069
:1005100008BD00BF9C02FF1F014BB3F8720070477B
:100520009C02FF1F014B9867012070479C02FF1F30
:10053000014B986F704700BF9C02FF1FB1F5803FD1
:100540000AD208B50E4A1278824210D00D4A1278AB
:10055000824203D0002008BD002070478BB20A4AB7
:100560001946A2F87630F8F7A9FC012008BD8BB235
:10057000054A1946A2F87430F8F7A0FC012008BD1E
:100580001100FF1F1200FF1F9C02FF1F084B1B786A
:10059000834208D0074B1B78834206BF064BB3F853
:1005A000760000207047044BB3F87400704700BF1A
:1005B0001100FF1F1200FF1F9C02FF1F014BD86795
:1005C000012070479C02FF1F014BD86F704700BF8E
:1005D0009C02FF1F014B1868704700BF7051FF1F3E
:1005E000014B1868704700BF6851FF1F014B186826
:1005F000704700BF6451FF1F014B1868704700BF70
:100600005C51FF1F014B1868704700BF6C51FF1F02
:10061000014B1868704700BF5051FF1F014B18680D
:10062000704700BF5851FF1F014B1868704700BF4B
:100630005451FF1F014B1868704700BF6051FF1FE6
:10064000014B1868704700BFCC12FF1F014B1860A8
:10065000704700BF7051FF1F014B1860704700BF0B
:100660006851FF1F014B1860704700BF6451FF1FA6
:10067000014B1860704700BF5C51FF1F014B1860B1
:10068000704700BF6C51FF1F014B1860704700BFDF
:100690005051FF1F014B1860704700BF5851FF1F9A
:1006A000014B1860704700BF5451FF1F014B186089
:1006B000704700BF6051FF1F014B1860704700BFBB
:1006C000CC12FF1F054B10B40022012418705C727D
:1006D0001A725960DA6010BC704700BF4C02FF1FED
:1006E000024B00225A721A72DA6070474C02FF1FE6
:1006F000014B187A704700BF4C02FF1F014B587A1C
:10070000704700BF4C02FF1F014BD868704700BF05
:100710004C02FF1F064BDA6801320021B2F57A7FE6
:10072000DA60196102D159721972D960704700BF3D
:100730004C02FF1FF0B4154D154E2C69366801347C
:1007400084B004AFB44207E90F002C6117DB2B7AA9
:10075000ABB1EB68B3F57A7F11DA1F010D4A009E49
:10076000D65101333A44019C02980399EB6000266C
:10077000B3F57A7F54609060D1602E6102D004B0EE
:10078000F0BC70476E722E72EE60F8E74C02FF1FED
:100790003C00FF1FD012FF1F4FF47A70704700BF5C
:1007A0004FF47A50704700BF04207047B0F57A7F4D
:1007B0000BDA032901DD0220704701EB8001044BB5
:1007C00053F821301360002070470120704700BFAC
:1007D000D012FF1F0A2807D8DFE800F00611150A1B
:1007E0000E0E060606060E00094B00225A617047DF
:1007F000074B03225A617047054B58617047044B01
:1008000001225A617047024B02225A61704700BFB1
:100810004C02FF1F014B5869704700BF4C02FF1F7D
:10082000014B1860704700BF3C00FF1F014B186868
:10083000704700BF3C00FF1F10B5144B1C78062CFE
:1008400008D8DFE804F00713171B1F0C04005A68D0
:10085000904207DD01221A7200225A7210BD5A68B6
:100860008242F7DC1A7A012AF6D010BD596891420B
:10087000F8DDEFE759688A42ECDCF3E75A688A4210
:10088000E8DCEFE75A689142E4DCEBE74C02FF1F3B
:10089000B0F5803F1DDBB0F1807F33DBB0F1805FCE
:1008A0003BDAB0F1806F3A4A4FDB0315D35C9B0112
:1008B0005A1C90FBF3F31A445210531C90FBF2F2B3
:1008C00013445B1003FB03F2904209DA013B184624
:1008D0007047FF2806DC002857DB2D4B1B5C1B09EB
:1008E00018467047B0F5805F294A26DBB0F5804F87
:1008F00041DB0312D35C013303FB03F29042E5DBDF
:1009000018467047B0F5801F214A0FDBB0F5800F05
:1009100029DB0314D25C1201CFE7B0F1804F18DB62
:100920001C4B98422CDD4FF6FF73D9E7B0F5802FB2
:100930001DDB0313D25C9200BFE7B0F5806F0DDBC7
:100940000311D35C9B080133D6E78314D35C5B01AE
:10095000AEE70F4A8315D35CDB01A9E78310D35CB4
:10096000DB080133C8E78313D25CD200A5E783120A
:10097000D25C5200A1E78311D35C5B080133BBE773
:10098000034A0316D35C1B0292E74FF0FF33A7E73D
:10099000E02701000080FE7FB0F5806F14D2B0F533
:1009A000007F08D2FF2895BF0A4B0B4BC018181ABE
:1009B00090F800017047B0F5407F07D3074B181A35
:1009C00090F800014042704700207047044BC05C23
:1009D00040427047E0270100DF290100DF2B0100C2
:1009E000E0260100904203DC8842B8BF0846704709
:1009F00010467047904203D8884238BF0846704777
:100A00001046704730B5DDE90345844275EB010EB1
:100A100007DB904271EB030400DB30BD1046194642
:100A200030BD2046294630BD70B514460E4600F054
:100A30008DFF0546204600F085FF04460146284606
:100A400001F08CF80146284600F0CAFE0546304603
:100A500000F07CFF214601F081F80146284600F0B5
:100A6000C1FE01F08DF970BD30B4029C0568E31A37
:100A70008A1A02FA03F32B44036043FA04F030BCF1
:100A8000704700BF44F6E612030C13FB02F3002B81
:100A900000B2B8BF03F5FF4310FB02F2B8BF7F33CB
:100AA000002A84B0B8BF02F5FF42C3F3CF33B8BF0A
:100AB0007F32ADF80C0003EBE2321344BDF80C209A
:100AC0005B4200209BB262F30F0063F31F4004B04F
:100AD000704700BFB0F90210B0F9003010B401FB4C
:100AE00001F20F4C03FB0322A24216D9120E3A3A2E
:100AF0000C4C34F8122002FB03F3002B02FB01F232
:100B0000BCBF03F5FF437F33002ABCBF02F5FF42A1
:100B10007F32DB13D2130380428010BC704700BFCA
:100B20000044FA3AE02901001F49B0F90020B1F968
:100B30000030B1F9021010B4B0F9024002FB03F02A
:100B40000028B8BF00F5FF4002FB01F204FB01F1F1
:100B5000B8BF7F300029B8BF01F5FF4103FB04F3A4
:100B6000B8BF7F31002B83B0B8BF03F5FF434FEA16
:100B7000E03000EBE131B8BF7F33002AB8BF02F5A7
:100B8000FF42ADF80410B8BF7F32BDF80410DB138C
:100B9000A3EBD23300209BB261F30F0063F31F403D
:100BA00003B010BC704700BF6402FF1FA0F50040F7
:100BB000C0F3891000F44073B3F5807F82B03FD05A
:100BC00029D9B3F5007F19D0B3F5407F35D1244B37
:100BD000C0B203EB4002400080F4FF70B2F88C20FA
:100BE00018445242B0F98C3012B292B200209BB23B
:100BF00062F30F0063F31F4002B07047C0B2184A9F
:100C0000430083F4FF73134402EB4000B3F98C20DC
:100C1000B0F98C30E9E783B9C0B2114A430083F4DC
:100C2000FF73134402EB4000B3F88C20B0F88C3013
:100C300052425B4212B21BB2D7E700231A46D4E7F6
:100C4000C0B2074A430083F4FF73134402EB400031
:100C5000B3F88C30B0F98C205B421BB2C5E700BF03
:100C6000E029010010B5044682B00846FFF79EFF58
:100C70001C4AB4F90030106002B203FB02F1B4F96F
:100C8000024000294FEA2040B8BF01F5FF4103FBB5
:100C900000F304FB00F0B8BF7F310028BCBF00F5B3
:100CA000FF407F30002BB8BF03F5FF4302FB04F287
:100CB0004FEAE131A1EBE030B8BF7F33002AADF855
:100CC0000400BCBF02F5FF427F32BDF80410DB1305
:100CD00003EBD23300209BB261F30F0063F31F409C
:100CE00002B010BD6402FF1F032923D8DFE801F022
:100CF0001C140C02104B400080F4FF701844B0F834
:100D00008C00404200B270470B4B03EB4000B0F840
:100D10008C00404200B27047074B400080F4FF70E7
:100D20001844B0F98C007047034B03EB4000B0F956
:100D30008C00704700207047E0290100002300224A
:100D4000C0E90223002303608361704770B5164C2D
:100D50002368C31A002BB8BF5B42B3F57A7F22DB4E
:100D6000054660680026FFF771FC6368E068A360D1
:100D70006660FFF771FCE36860692361E660FFF776
:100D800071FCA0696661FFF773FCE069A661FFF77B
:100D900075FCE369606A2362E661FFF775FC636ACC
:100DA00025606662A36270BD6802FF1F024A536835
:100DB00001335360704700BF6802FF1F014B586842
:100DC000704700BF6802FF1F014B9868704700BF63
:100DD0006802FF1F024AD3680133D360704700BF27
:100DE0006802FF1F014B1869704700BF6802FF1FB0
:100DF000024A536901335361704700BF6802FF1F05
:100E0000024A936901339361704700BF6802FF1F74
:100E1000024AD3690133D361704700BF6802FF1FE4
:100E2000014B186A704700BF6802FF1F024BD86968
:100E300000EB8000400070476802FF1F024A536ABF
:100E400001335362704700BF6802FF1F014B986A6D
:100E5000704700BF6802FF1F024B586A00EB80001A
:100E6000400070476802FF1F81F0004102E000BFB0
:100E700083F0004330B54FEA41044FEA430594EA5A
:100E8000050F08BF90EA020F1FBF54EA000C55EA95
:100E9000020C7FEA645C7FEA655C00F0E2804FEA66
:100EA0005454D4EB5555B8BF6D420CDD2C4480EA48
:100EB000020281EA030382EA000083EA010180EA78
:100EC000020281EA0303362D88BF30BD11F0004FC6
:100ED0004FEA01314FF4801C4CEA113102D04042FC
:100EE00061EB410113F0004F4FEA03334CEA133337
:100EF00002D0524263EB430394EA050F00F0A7804F
:100F0000A4F10104D5F1200E0DDB02FA0EFC22FA49
:100F100005F2801841F1000103FA0EF2801843FA3D
:100F200005F359410EE0A5F120050EF1200E012A2E
:100F300003FA0EFC28BF4CF0020C43FA05F3C0186C
:100F400051EBE37101F0004507D54FF0000EDCF1E5
:100F5000000C7EEB00006EEB0101B1F5801F1BD38E
:100F6000B1F5001F0CD349085FEA30004FEA3C0C92
:100F700004F101044FEA445212F5800F80F09A8088
:100F8000BCF1004F08BF5FEA500C50F1000041EB8C
:100F9000045141EA050130BD5FEA4C0C404141EB90
:100FA000010111F4801FA4F10104E9D191F0000FB7
:100FB00004BF01460020B1FA81F308BF2033A3F13A
:100FC0000B03B3F120020CDA0C3208DD02F1140C31
:100FD000C2F10C0201FA0CF021FA02F10CE002F16C
:100FE0001402D8BFC2F1200C01FA02F120FA0CFC65
:100FF000DCBF41EA0C019040E41AA2BF01EB0451AE
:10100000294330BD6FEA04041F3C1CDA0C340EDCAB
:1010100004F11404C4F1200220FA04F001FA02F3EE
:1010200040EA030021FA04F345EA030130BDC4F1AC
:101030000C04C4F1200220FA02F001FA04F340EAA1
:101040000300294630BD21FA04F0294630BD94F052
:10105000000F83F4801306BF81F480110134013D39
:101060004EE77FEA645C18BF7FEA655C29D094EAAA
:10107000050F08BF90EA020F05D054EA000C04BF28
:101080001946104630BD91EA030F1EBF0021002013
:1010900030BD5FEA545C05D14000494128BF41F0B2
:1010A000004130BD14F580043CBF01F5801130BD16
:1010B00001F0004545F0FE4141F470014FF00000A1
:1010C00030BD7FEA645C1ABF194610467FEA655C52
:1010D0001CBF0B46024650EA013406BF52EA0335F4
:1010E00091EA030F41F4002130BD00BF90F0000FE2
:1010F00004BF0021704730B54FF4806404F132041E
:101100004FF000054FF0000150E700BF90F0000FD6
:1011100004BF0021704730B54FF4806404F13204FD
:1011200010F0004548BF40424FF000013EE700BFCD
:1011300042004FEAE2014FEA31014FEA02701FBF5D
:1011400012F07F4393F07F4F81F06051704792F02F
:10115000000F14BF93F07F4F704730B54FF46074A9
:1011600001F0004521F0004120E700BF50EA0102F4
:1011700008BF704730B54FF000050AE050EA0102A1
:1011800008BF704730B511F0004502D5404261EB11
:1011900041014FF4806404F132045FEA915C3FF452
:1011A000DCAE4FF003025FEADC0C18BF03325FEAEB
:1011B000DC0C18BF033202EBDC02C2F1200300FAA0
:1011C00003FC20FA02F001FA03FE40EA0E0021FAC5
:1011D00002F11444C1E600BF70B54FF0FF0C4CF4AF
:1011E000E06C1CEA11541DBF1CEA135594EA0C0F65
:1011F00095EA0C0F00F0DEF82C4481EA030621EAA0
:101200004C5123EA4C5350EA013518BF52EA0335DA
:1012100041F4801143F4801338D0A0FB02CE4FF08C
:101220000005E1FB02E506F00042E0FB03E54FF0BC
:101230000006E1FB03569CF0000F18BF4EF0010EB4
:10124000A4F1FF04B6F5007F64F5407404D25FEAB0
:101250004E0E6D4146EB060642EAC62141EA555163
:101260004FEAC52040EA5E504FEACE2EB4F1FD0CA5
:1012700088BFBCF5E06F1ED8BEF1004F08BF5FEA23
:10128000500E50F1000041EB045170BD06F00046D5
:1012900046EA010140EA020081EA0301B4EB5C0482
:1012A000C2BFD4EB0C0541EA045170BD41F480117A
:1012B0004FF0000E013C00F3AB8014F1360FDEBF9F
:1012C000002001F0004170BDC4F10004203C35DA7B
:1012D0000C341BDC04F11404C4F1200500FA05F3FE
:1012E00020FA04F001FA05F240EA020001F000429F
:1012F00021F0004110EBD37021FA04F642EB060115
:101300005EEA430E08BF20EAD37070BDC4F10C043E
:10131000C4F1200500FA04F320FA05F001FA04F202
:1013200040EA020001F0004110EBD37041F10001EE
:101330005EEA430E08BF20EAD37070BDC4F12005F9
:1013400000FA05F24EEA020E20FA04F301FA05F261
:1013500043EA020321FA04F001F0004121FA04F209
:1013600020EA020000EBD3705EEA430E08BF20EAD9
:10137000D37070BD94F0000F0FD101F00046400013
:1013800041EB010111F4801F08BF013CF7D041EA95
:10139000060195F0000F18BF704703F00046520099
:1013A00043EB030313F4801F08BF013DF7D043EA6A
:1013B0000603704794EA0C0F0CEA135518BF95EA20
:1013C0000C0F0CD050EA410618BF52EA4306D1D1A7
:1013D00081EA030101F000414FF0000070BD50EAC6
:1013E000410606BF1046194652EA430619D094EA50
:1013F0000C0F02D150EA013613D195EA0C0F05D13A
:1014000052EA03361CBF104619460AD181EA03018D
:1014100001F0004141F0FE4141F470014FF0000045
:1014200070BD41F0FE4141F4780170BD70B54FF0E0
:10143000FF0C4CF4E06C1CEA11541DBF1CEA135560
:1014400094EA0C0F95EA0C0F00F0A7F8A4EB050442
:1014500081EA030E52EA03354FEA013100F0888039
:101460004FEA03334FF0805545EA131343EA126302
:101470004FEA022245EA111545EA10654FEA0026B7
:101480000EF000419D4208BF964244F1FD0404F570
:10149000407402D25B084FEA3202B61A65EB0305CC
:1014A0005B084FEA32024FF480104FF4002CB6EB89
:1014B000020E75EB030E22BFB61A754640EA0C0009
:1014C0005B084FEA3202B6EB020E75EB030E22BF49
:1014D000B61A754640EA5C005B084FEA3202B6EB8A
:1014E000020E75EB030E22BFB61A754640EA9C0049
:1014F0005B084FEA3202B6EB020E75EB030E22BF19
:10150000B61A754640EADC0055EA060E18D04FEAD6
:10151000051545EA16754FEA06164FEAC30343EA76
:1015200052734FEAC2025FEA1C1CC0D111F4801F43
:101530000BD141EA00014FF000004FF0004CB6E73C
:1015400011F4801F04BF01430020B4F1FD0C88BFDB
:10155000BCF5E06F3FF6AFAEB5EB030C04BFB6EBE6
:10156000020C5FEA500C50F1000041EB045170BDD9
:101570000EF0004E4EEA113114EB5C04C2BFD4EB06
:101580000C0541EA045170BD41F480114FF0000E8A
:10159000013C90E645EA060E8DE60CEA135594EA06
:1015A0000C0F08BF95EA0C0F3FF43BAF94EA0C0F09
:1015B0000AD150EA01347FF434AF95EA0C0F7FF47E
:1015C00025AF104619462CE795EA0C0F06D152EAD2
:1015D00003353FF4FDAE1046194622E750EA4106B6
:1015E00018BF52EA43067FF4C5AE50EA41047FF4C7
:1015F0000DAF52EA43057FF4EBAE12E74FF0FF3C2C
:1016000006E000BF4FF0010C02E000BF4FF0010CFC
:101610004DF804CD4FEA410C7FEA6C5C4FEA430C75
:1016200018BF7FEA6C5C1BD001B050EA410C0CBFC4
:1016300052EA430C91EA030F02BF90EA020F002026
:10164000704710F1000F91EA030F58BF994208BF8D
:1016500090422CBFD8176FEAE37040F0010070474A
:101660004FEA410C7FEA6C5C02D150EA013C07D1A1
:101670004FEA430C7FEA6C5CD6D152EA033CD3D0EC
:101680005DF8040B704700BF8446104662468C46E6
:101690001946634600E000BF01B5FFF7B7FF002819
:1016A00048BF10F1000F01BD4DF808EDFFF7F4FF42
:1016B0000CBF012000205DF808FB00BF4DF808EDCD
:1016C000FFF7EAFF34BF012000205DF808FB00BFF0
:1016D0004DF808EDFFF7E0FF94BF012000205DF812
:1016E00008FB00BF4DF808EDFFF7CEFF94BF0120C7
:1016F00000205DF808FB00BF4DF808EDFFF7C4FFC0
:1017000034BF012000205DF808FB00BF4FEA410C08
:101710007FEA6C5C02D150EA013C0AD14FEA430CEB
:101720007FEA6C5C02D152EA033C02D14FF0000028
:1017300070474FF0010070474FEA4102B2F1E043B9
:1017400024BFB3F5001CDCF1FE5C0DD901F0004CA8
:101750004FEAC0024CEA5070B2F1004F40EB8300F8
:1017600008BF20F00100704711F0804F21D113F124
:101770003872BCBF01F00040704741F480114FEA5D
:101780005252C2F11802C2F1200C10FA0CF320FAE6
:1017900002F018BF40F001004FEAC1234FEAD32303
:1017A00003FA0CFC40EA0C0023FA02F34FEA43036D
:1017B000CCE77FEA625307D150EA01331EBF4FF0F6
:1017C000FE4040F44000704701F0004040F0FE4011
:1017D00040F40000704700BF80F0004002E000BF0E
:1017E00081F0004142001FBF5FEA410392EA030F0C
:1017F0007FEA226C7FEA236C6AD04FEA1262D2EB56
:101800001363C1BFD218414048404140B8BF5B425A
:10181000192B88BF704710F0004F40F4000020F0F3
:101820007F4018BF404211F0004F41F4000121F009
:101830007F4118BF494292EA030F3FD0A2F1010253
:1018400041FA03FC10EB0C00C3F1200301FA03F191
:1018500000F0004302D5494260EB4000B0F5000FB4
:1018600013D3B0F1807F06D340084FEA310102F173
:101870000102FE2A51D2B1F1004F40EBC25008BF25
:1018800020F0010040EA03007047490040EB0000EF
:1018900010F4000FA2F10102EDD1B0FA80FCACF11E
:1018A000080CB2EB0C0200FA0CF0AABF00EBC2501D
:1018B00052421843BCBFD0401843704792F0000F0B
:1018C00081F4000106BF80F400000132013BB5E75E
:1018D0004FEA41037FEA226C18BF7FEA236C21D0D4
:1018E00092EA030F04D092F0000F08BF0846704739
:1018F00090EA010F1CBF0020704712F07F4F04D107
:10190000400028BF40F00040704712F100723CBF19
:1019100000F50000704700F0004343F0FE4040F443
:10192000000070477FEA226216BF08467FEA236301
:101930000146420206BF5FEA412390EA010F40F4EC
:10194000800070474FF0000304E000BF10F0004338
:1019500048BF40425FEA000C08BF704743F096431F
:1019600001464FF000001CE050EA010208BF70473A
:101970004FF000030AE000BF50EA010208BF7047C1
:1019800011F0004302D5404261EB41015FEA010CD6
:1019900002BF84460146002043F0B64308BFA3F1CE
:1019A0008053A3F50003BCFA8CF2083AA3EBC253B0
:1019B00010DB01FA02FC634400FA02FCC2F12002CF
:1019C000BCF1004F20FA02F243EB020008BF20F006
:1019D0000100704702F1200201FA02FCC2F120026C
:1019E00050EA4C0021FA02F243EB020008BF20EA61
:1019F000DC7070474FF0FF0C1CEAD0521EBF1CEA8F
:101A0000D15392EA0C0F93EA0C0F6FD01A4480EA7C
:101A1000010C400218BF5FEA41211ED04FF0006365
:101A200043EA501043EA5111A0FB01310CF0004091
:101A3000B1F5000F3EBF490041EAD3715B0040EAB7
:101A4000010062F17F02FD2A1DD8B3F1004F40EB87
:101A5000C25008BF20F00100704790F0000F0CF05A
:101A6000004C08BF49024CEA502040EA51207F3A1E
:101A7000C2BFD2F1FF0340EAC250704740F40000F9
:101A80004FF00003013A5DDC12F1190FDCBF00F0EA
:101A900000407047C2F10002410021FA02F1C2F198
:101AA000200200FA02FC5FEA310040F1000053EA34
:101AB0004C0308BF20EADC70704792F0000F00F082
:101AC000004C02BF400010F4000F013AF9D040EA88
:101AD0000C0093F0000F01F0004C02BF490011F41C
:101AE000000F013BF9D041EA0C018FE70CEAD1531A
:101AF00092EA0C0F18BF93EA0C0F0AD030F0004C9A
:101B000018BF31F0004CD8D180EA010000F000404D
:101B1000704790F0000F17BF90F0004F084691F00B
:101B2000000F91F0004F14D092EA0C0F01D1420245
:101B30000FD193EA0C0F03D14B0218BF084608D10E
:101B400080EA010000F0004040F0FE4040F4000058
:101B5000704740F0FE4040F4400070474FF0FF0CEB
:101B60001CEAD0521EBF1CEAD15392EA0C0F93EA32
:101B70000C0F69D0A2EB030280EA010C49024FEA84
:101B8000402037D04FF0805343EA111143EA10133D
:101B90000CF000408B4238BF5B0042F17D024FF4F5
:101BA000000C8B4224BF5B1A40EA0C00B3EB510FD0
:101BB00024BFA3EB510340EA5C00B3EB910F24BFB9
:101BC000A3EB910340EA9C00B3EBD10F24BFA3EB3E
:101BD000D10340EADC001B0118BF5FEA1C1CE0D106
:101BE000FD2A3FF650AF8B4240EBC25008BF20F0B9
:101BF000010070470CF0004C4CEA50207F32C2BF0D
:101C0000D2F1FF0340EAC250704740F400004FF0A9
:101C10000003013A37E792F0000F00F0004C02BFDA
:101C2000400010F4000F013AF9D040EA0C0093F0A4
:101C3000000F01F0004C02BF490011F4000F013BFE
:101C4000F9D041EA0C0195E70CEAD15392EA0C0F66
:101C500008D142027FF47DAF93EA0C0F7FF470AF9E
:101C6000084676E793EA0C0F04D14B023FF44CAFE1
:101C700008466EE730F0004C18BF31F0004CCAD176
:101C800030F000427FF45CAF31F000437FF43CAFB2
:101C90005FE700BF4FF0FF3C06E000BF4FF0010CD4
:101CA00002E000BF4FF0010C4DF804CD4FEA4002B6
:101CB0004FEA41037FEA226C18BF7FEA236C11D000
:101CC00001B052EA530C18BF90EA010F58BFB2EBB3
:101CD000030088BFC81738BF6FEAE17018BF40F033
:101CE000010070477FEA226C02D15FEA402C05D1E7
:101CF0007FEA236CE4D15FEA412CE1D05DF8040B6C
:101D0000704700BF844608466146FFE70FB5FFF7FE
:101D1000C9FF002848BF10F1000F0FBD4DF808EDB6
:101D2000FFF7F4FF0CBF012000205DF808FB00BFA7
:101D30004DF808EDFFF7EAFF34BF012000205DF801
:101D400008FB00BF4DF808EDFFF7E0FF94BF01204E
:101D500000205DF808FB00BF4DF808EDFFF7D2FF4B
:101D600094BF012000205DF808FB00BF4DF808ED8E
:101D7000FFF7C8FF34BF012000205DF808FB00BF5B
:101D80004FEA4002B2F1FE4F0FD34FF09E03B3EB88
:101D900012620DD94FEA002343F0004310F0004FC8
:101DA00023FA02F018BF404270474FF0000070471E
:101DB00012F1610F01D1420205D110F0004008BFBD
:101DC0006FF0004070474FF0000070477BB972B968
:101DD0000029BEBF00204FF0004106E008BF0028E8
:101DE0001CBF6FF000414FF0FF3000F0FFB9ADF1C4
:101DF000080C6DE904CE002909DB002B1ADB00F08A
:101E000087F8DDF804E0DDE9022304B070474042C2
:101E100061EB4101002B1BDB00F07AF8DDF804E0F8
:101E2000DDE9022304B0404261EB4101524263EB21
:101E300043037047524263EB430300F069F8DDF857
:101E400004E0DDE9022304B0404261EB4101704748
:101E5000524263EB430300F05BF8DDF804E0DDE998
:101E6000022304B0524263EB4303704753B94AB9AB
:101E7000002908BF00281CBF4FF0FF314FF0FF3092
:101E800000F0B4B9ADF1080C6DE904CE00F040F8F3
:101E9000DDF804E0DDE9022304B0704710B500214D
:101EA0000446FFF745FF20B92046BDE8104000F08A
:101EB00009B804F1004000F005F8404261EB41012F
:101EC00010BD00BFD0B5FFF733F900220E4B064618
:101ED0000F46FFF781F900F08BF90446FFF706F98A
:101EE00000220A4BFFF778F902460B463046394686
:101EF000FEF7BEFF00F07CF92346002242EA000212
:101F000010461946D0BD00BF0000F03D0000F04172
:101F10002DE9F0478C460D460446089E002B51D112
:101F20008A4217466DD9B2FA82FEBEF1000F0BD07D
:101F3000CEF1200C01FA0EF520FA0CFC02FA0EF795
:101F40004CEA050C00FA0EF44FEA174A250CBCFBCC
:101F5000FAF81FFA87F90AFB18CC45EA0C4508FB8A
:101F600009F3AB420AD9ED1908F1FF3280F0238161
:101F7000AB4240F22081A8F102083D44ED1AA4B220
:101F8000B5FBFAF00AFB105544EA054400FB09F9D9
:101F9000A14509D9E41900F1FF3380F00A81A14578
:101FA00040F2078102383C44A4EB090440EA0840AF
:101FB0000021002E61D024FA0EF4002334607360F7
:101FC000BDE8F0878B4207D9002E54D0002186E867
:101FD00021000846BDE8F087B3FA83F1002940F0FC
:101FE0008E80AB4202D3824200F2FA80841A65EB03
:101FF00003050120AC46002E3FD086E81010BDE856
:10200000F08712B90127B7FBF2F7B7FA87FEBEF1E6
:10201000000F34D1EB1B3A0C1FFA87FC0121B3FBF4
:10202000F2F8250C02FB183345EA03450CFB08F3D4
:10203000AB4207D9ED1908F1FF3002D2AB4200F2F2
:10204000D1808046ED1AA3B2B5FBF2F002FB105529
:1020500043EA05440CFB00FCA44507D9E41900F150
:10206000FF3302D2A44500F2B8801846A4EB0C045A
:1020700040EA08409DE731463046BDE8F087CEF1A2
:10208000200405FA0EF307FA0EF720FA04F83A0CCA
:1020900025FA04F448EA0308B4FBF2F14FEA1845C4
:1020A00002FB11441FFA87FC45EA044501FB0CF3CF
:1020B000AB4200FA0EF409D9ED1901F1FF3080F0BE
:1020C0008A80AB4240F2878002393D44EB1A1FFA06
:1020D00088F5B3FBF2F002FB103345EA034500FB41
:1020E0000CF3AB4207D9ED1900F1FF386FD2AB42C8
:1020F0006DD902383D44EB1A40EA01418FE7C1F146
:10210000200722FA07F88B4005FA01F448EA030396
:1021100020FA07FE4FEA134CFD404EEA040EB5FBD1
:10212000FCF94FEA1E440CFB19551FFA83F844EAE8
:10213000054509FB08F4AC4202FA01F200FA01FA83
:1021400008D9ED1809F1FF3043D2AC4241D9A9F1C9
:1021500002091D442D1B1FFA8EFEB5FBFCF00CFB83
:1021600010554EEA054400FB08F8A04507D9E418CD
:1021700000F1FF3529D2A04527D902381C4440EA96
:102180000940A4EB0804A0FB02894C45C6464D4615
:1021900015D312D056B1BAEB0E0364EB050404FA62
:1021A00007F7CB401F43CC40376074600021BDE887
:1021B000F0871846F8E69046E0E6C245EAD2B8EB6A
:1021C000020E69EB03050138E4E72846D7E74046ED
:1021D00091E78146BEE7014678E702383C4445E78F
:1021E000084608E7A8F102083D442BE7704700BF06
:1021F0004A0011D212F5001211D20DD56FF4787386
:10220000B3EB62520ED44FEAC12343F0004343EADA
:10221000505323FA02F070474FF00000704750EA25
:10222000013002D14FF0FF3070474FF0000070478F
:1022300038B5F7F703FC62B6F6F70CFBF6F728FBA8
:10224000F6F78CFB184C0546F7F7FAFBF7F710F892
:102250002A4616492046F8F7D9F82078F7F79AF970
:102260002079F7F7E1F960792189228AF6F7C6FE2D
:10227000F6F704FCF6F766FE0D4B01221A70F9F72B
:10228000C9FEFCF73FFE40F21670F8F72DFF012063
:10229000FCF7E0F9FDF7EEF8FEF788FDF7F7E4FB51
:1022A000FEF754FDF3E700BF2003FF1F9C02FF1F52
:1022B0001C03FF1F2DE970438AB004460D4600F051
:1022C00077F8354B93F90060731C804689460DD032
:1022D00022462B4620462946FFF718FA30B900223D
:1022E000002320462946FFF707FA20B14046494619
:1022F0000AB0BDE87083294B0890CDE90245CDE9CD
:102300000445019320462946CEB9254D4FF060443F
:1023100000220023CDE90645FFF7C6F9002833D097
:1023200002230093684600F037FAA8B1089BC3B9AE
:10233000DDE90689404649460AB0BDE87083194D7B
:10234000002400220023CDE90645FFF7ADF968B16E
:1023500002239E420093E5D100F026FA2223036077
:10236000E4E700F021FA089B0360E1E70123022E75
:1023700000930BD100F018FA212303600A4800F003
:102380000DFACDE90601D1E701230093684600F07C
:1023900003FA0028F2D1EDE7A400FF1F802C010012
:1023A000FFFFEFC70000F0FF702C010000000000ED
:1023B0002DE9F04FB1F5801F85B006460F460B465C
:1023C0005ADA024621F00044224300F0F880002946
:1023D000C0F27A810022D64BFEF7FEFED54A0B46AC
:1023E000934206460F466FF0350C4ADCC3F31305E3
:1023F00005F5152E0EF6647E0EF4801E8EF07F52CB
:1024000082F440121C1542EA0507A4F2FF3464442A
:102410000022C94B3046394604EB1E54FEF728FD16
:10242000AB1CC3F31303022B82468B464FF0000212
:1024300030DC0023FFF738F9002800F0C980002CB9
:1024400000F04B812046FEF761FEA5A3D3E90023EF
:1024500006460F46FEF7C0FEA3A3D3E900230446B9
:102460000D4630463946FEF7B7FE02460B4620467B
:102470002946FEF7FFFC0AE0AE4A93424FF0000CFB
:10248000B4DD32463B4630463946FEF7F3FC05B034
:10249000BDE8F08F4FF08043FEF7ECFC02460B46A0
:1024A00050465946FEF7C2FF064620460F46FEF745
:1024B0002DFE3246CDE900013B4630463946CDE996
:1024C0000267FEF789FE02460B4680468946FEF704
:1024D00083FE87A3D3E9002306460F46FEF77CFE62
:1024E00085A3D3E90023FEF7C5FC32463B46FEF741
:1024F00073FE83A3D3E90023FEF7BCFC32463B46C0
:10250000FEF76AFE80A3D3E90023FEF7B3FC424640
:102510004B46FEF761FE7EA3D3E900238046894641
:1025200030463946FEF758FE7BA3D3E90023FEF779
:10253000A1FC32463B46FEF74FFE79A3D3E90023C8
:10254000FEF798FC32463B46FEF746FE0B46024637
:1025500049464046FEF78EFCA5F5C223C5F5D725B2
:10256000A3F27A4351351D43002D8046894656DD3E
:102570000022724B50465946FEF72EFE52465B46ED
:10258000FEF72AFE06460F46002C68D132463B462F
:1025900040464946FEF76EFCDDE90223FEF71CFECD
:1025A00002460B4630463946FEF762FC02460B46B1
:1025B00050465946FEF75CFC05B0BDE8F08F00229E
:1025C000002300205E49FEF731FF05B0BDE8F08F23
:1025D00055A3D3E9002350465946FEF7FDFD0246B8
:1025E0000B4600205549FEF743FC524606460F466F
:1025F0005B4650465946FEF7EFFD02460B46304615
:102600003946FEF7E9FD06460F46002C40F09A8059
:1026100002460B4650465946FEF72AFC37E7002C87
:1026200000F0A4802EA3D3E90023DDE90001FEF72A
:10263000D3FD42464B4604460D4650465946FEF7EA
:1026400017FCDDE90223FEF7C7FD27A3D3E900232A
:1026500006460F46DDE90001FEF7BEFD21E020A39E
:10266000D3E90023DDE90001FEF7B6FD32463B4623
:1026700004460D4640464946FEF7FCFBDDE90223D1
:10268000FEF7AAFD18A3D3E9002380468946DDE9B9
:102690000001FEF7A1FD02460B4640464946FEF703
:1026A000E9FB02460B4630463946FEF7E1FB52464F
:1026B0005B46FEF7DDFB02460B4620462946FEF749
:1026C000D7FB05B0BDE8F08F02460B46FEF7D0FB06
:1026D00000220023FEF7AAFED9E600200021D6E65C
:1026E0000000E0FE422EE63F763C7935EF39EA3DC8
:1026F00044523EDF12F1C23FDE03CB966446C73F31
:10270000599322942449D23F935555555555E53F49
:102710009FC678D0099AC33FAF788E1DC571CC3F54
:1027200004FA97999999D93F555555555555D53F1F
:1027300000005043FFFFEF7F0000F03F0000E03F4C
:10274000000050C32046FEF7E1FC0FA3D3E90023AD
:1027500080468946FEF740FD0DA3D3E900230446D9
:102760000D4640464946FEF737FD9AE702460B46BE
:1027700050465946FEF77CFBDDE90223FEF72CFDAF
:1027800014E700BFAFF300800000E0FE422EE63FFA
:10279000763C7935EF39EA3D002070470020014949
:1027A000704700BF0000F87F014B1868704700BFFA
:1027B0004000FF1F8025000040380000004B000053
:1027C000807000000096000000E10000002C010075
:1027D00000C201005515AC6A004001C0ABEA579534
:1027E0000010161B2023272A2D30323537393B3D68
:1027F0004041434547494B4C4E505153545657590D
:102800005A5B5D5E60616263656667686A6B6C6D8A
:102810006E707172737475767778797A7B7C7D7E51
:1028200080808182838485868788898A8B8C8D8E3F
:102830008F9090919293949596969798999A9B9B46
:102840009C9D9E9FA0A0A1A2A3A3A4A5A6A7A7A864
:10285000A9AAAAABACADADAEAFB0B0B1B2B2B3B491
:10286000B5B5B6B7B7B8B9B9BABBBBBCBDBDBEBFCD
:10287000C0C0C1C1C2C3C3C4C5C5C6C7C7C8C9C912
:10288000CACBCBCCCCCDCECECFD0D0D1D1D2D3D35E
:10289000D4D4D5D6D6D7D7D8D9D9DADADBDBDCDDB4
:1028A000DDDEDEDFE0E0E1E1E2E2E3E3E4E5E5E610
:1028B000E6E7E7E8E8E9EAEAEBEBECECEDEDEEEE73
:1028C000EFF0F0F1F1F2F2F3F3F4F4F5F5F6F6F7D8
:1028D000F7F8F8F9F9FAFAFBFBFCFCFDFDFEFEFF48
:1028E000000203050608090B0D0E1011131416172C
:1028F000191B1C1E1F2122242527292A2C2D2F308D
:102900003233353638393B3C3E3F414344464749F4
:102910004A4C4D4F505153545657595A5C5D5F6065
:102920006263646667696A6C6D6E707173747577E3
:10293000787A7B7C7E7F808283848687888A8B8C72
:102940008E8F90929394959798999A9C9D9E9FA113
:10295000A2A3A4A5A7A8A9AAABACAEAFB0B1B2B3CD
:10296000B4B5B7B8B9BABBBCBDBEBFC0C1C2C3C4A1
:10297000C5C6C7C8C9CACBCCCDCECFD0D0D1D2D393
:10298000D4D5D6D7D7D8D9DADBDCDCDDDEDFDFE0A3
:10299000E1E2E2E3E4E4E5E6E7E7E8E8E9EAEAEBD6
:1029A000ECECEDEDEEEEEFF0F0F1F1F2F2F3F3F42A
:1029B000F4F4F5F5F6F6F7F7F7F8F8F8F9F9F9FAA7
:1029C000FAFAFBFBFBFCFCFCFCFCFDFDFDFDFDFE47
:1029D000FEFEFEFEFEFEFFFFFFFFFFFFFFFFFFFF0D
:1029E0006B7FD87EB87DA07C8F7B857A8279857855
:1029F0000878147726763D7559747B73A172367208
:102A000064719670CC6F076F456EE66D2A6D726CBF
:102A1000BE6B0D6B5F6AB5696169BB6819687967E0
:102A2000DC664266AB656065CC643B64AD63206385
:102A300096620F62CB614761C4604460C65F495FC4
:102A4000CE5E925E1A5EA45D2F5DBD5C4B5CDC5B6E
:102A5000A55B385BCC5A625AF95992592C59F958EE
:102A600095583358D15771571257B4560000C900C2
:102A700092015B022403ED03B6047F0548061107AB
:102A8000D907A2086A09330AFB0AC40B8C0C540D3F
:102A90001C0EE30EAB0F72103A110112C8128F1305
:102AA00055141C15E215A8166E173318F918BE191F
:102AB000821A471B0B1CCF1C931D571E1A1FDD1FAC
:102AC0009F2061212322E522A62367242825E825CB
:102AD000A82667272628E528A329612A1F2BDC2B97
:102AE000992C552D112ECC2E872F4130FB30B5312E
:102AF0006E322633DF3396344D350436BA366F37AF
:102B00002438D9388C39403AF23AA53B563C073D37
:102B1000B83D683E173FC53F73402141CE417A42E0
:102B20002543D0437A442445CD4575461C47C347C9
:102B300069480F49B449584AFB4A9D4B3F4CE04C09
:102B4000814D204EBF4E5D4FFB4F97503351CE51BC
:102B5000685202539B533254C9546055F5558A56F6
:102B60001D57B0574258D3586459F359825A0F5BD6
:102B70009C5B285CB35C3E5DC75D4F5ED75E5D5F6E
:102B8000E35F6860EB606E61F0617162F1627063D7
:102B9000EE636C64E8646365DD655666CF66466720
:102BA000BC673268A66819698B69FD696D6ADC6A61
:102BB0004A6BB76B236C8E6CF86C616DC96D306EAF
:102BC000966EFB6E5E6FC16F22708370E270407113
:102BD0009D71F9715472AE7207735E73B5730A74A6
:102BE0005F74B27404755575A575F37541768D766D
:102BF000D87622776B77B377FA773F788478C7787F
:102C000009794A798979C879057A417A7C7AB67ADC
:102C1000EE7A267B5C7B917BC57BF87B297C597C9B
:102C2000887CB67CE37C0E7D397D627D897DB07DBC
:102C3000D57DFA7D1D7E3E7E5F7E7E7E9C7EB97E4A
:102C4000D57EEF7E097F217F377F4D7F617F747F47
:102C5000867F977FA67FB47FC17FCD7FD87FE17FBE
:102C6000E97FF07FF57FF97FFD7FFE7F56312E31C2
:102C70000000000043313630563231310000000090
:102C80006C6F6700F8B500BFF8BC08BC9E46704783
:0C2C9000F8B500BFF8BC08BC9E467047B9
:102C9C00F0B472B6114B70221A701A781206FCD569
:102CAC00C0F30744C0F307220625DD710F0E9C719B
:102CBC00C1F307465A71C1F30725C0B2C9B28024CB
:102CCC00064A1871DF729E725D7219721C7013784D
:102CDC001B06FCD562B6F0BC704700BF000002407A
:082CEC0024F2FF7F010000004B
:042CF4003584000023
:042CF8001184000043
:102CFC00010501010105070D010203003200050465
:102D0C006C2C0100742C0100010000C0FE7FFFFF41
:102D1C00014001000000803F0000803F01000000E6
:102D2C00FF000000010000004400FF1F0000000035
:102D3C000000000000000000000000000000000087
:102D4C000000000000000000000000000000000077
:102D5C000000000000000000000000000000000067
:102D6C000000000000000000000000000000000057
:102D7C000000000000000000000000000000000047
:102D8C000000000000000000000000000100000036
:102D9C00FC2C01000800FF1FA00000000000000038
:082DAC0000000000000000001F
:020000020000FC
:020000041FFFDC
:0400000000000000FC
:04000003000087BDB5
:00000001FF
